:020000040000FA
:06000000D1EF34F0120004
:0600080080EF2EF0120053
:06002A0006003A6A000026
:100030007503000004000000186A0000960200002A
:1000400022000000F06900006E020000280000009D
:10005000EE690000FD01000002000000EC690000F4
:10006000FE00000002000000DC6900002D0300001B
:04007000100000007C
:0C0074000B01006B0A0E005D26E200513B
:10008000220DF3CF01FBF4CF02FB000E01270C0E73
:100090000223DFEC08F0EF6A34EC0AF0EF9034EC66
:1000A0000AF0EF8234EC0AF0EF8434EC0AF0EF98B7
:1000B00034EC0AF0EF96DFEC08F0EFEC09F0DFEC3F
:1000C00008F003EC0AF0002BD7D70101496B040EAE
:1000D0004A6F4B6B4C6B4D6B4E6B12000B01006B00
:1000E0000A0E005D36E20051220DF3CF01FBF4CF82
:1000F00002FB000E01270C0E0223CEEC08F0EF509D
:10010000000925E1CEEC08F0010EEF6ECEEC08F010
:100110000B0E4FC1EBFF0C0E50C1EBFFCEEC08F005
:100120000D0EEB6A0E0EEB6ACEEC08F0FFEC09F058
:1001300046EC0AF0EF8046EC0AF0EF96CEEC08F0C1
:10014000EFEC09F046EC0AF0EF8200511200002BB0
:10015000C7D7FE0C0B016F6B6C6B0A0E6C5D14E263
:100160006C51220DF3CF6DFBF4CF6EFB000E6D27AB
:100170000C0E6E2385EC08F0EF50000903E1010E30
:100180006F6F02D06C2BE9D76F5101E1FE0C0101BA
:10019000492B000E4A2385EC08F00B0E49C1EBFFFA
:1001A0000C0E4AC1EBFF880ED8804955130E4A55F4
:1001B00003E2496B040E4A6F85EC08F0A1EC09F0EC
:1001C000EF9085EC08F00D0E53C1EBFF0E0E54C1FD
:1001D000EBFF4B2B000E4C234D234E2307EC0AF074
:1001E00043EC09F085EC08F0180E6DEC08F067ECB4
:1001F00009F00A0EE66EE66A51C1E6FF52C1E6FF5B
:1002000085EC08F08FEC08F0F9EC08F00101020E23
:100210007E6F85EC08F0F3EC09F007EC0AF0E9ECEE
:1002200008F085EC08F0F7EC09F085EC08F0FBEC41
:1002300009F085EC08F0D8EC08F085EC08F0030E26
:10024000EF6E07EC0AF093EC09F085EC08F0F2ECA5
:1002500008F00B016C51120001015551A8EC08F097
:10026000EF50040801E0000C010C01015651220D71
:10027000F3CF81FBF4CF82FB000E0B0181270C0E24
:100280008223E4EC08F0EF50040806E081CB88F10B
:1002900082CB89F1CCEF06F056C160F14CD9F9EC74
:1002A00008F00101110E7E6FE4EC08F0F3EC09F0A8
:1002B000E4EC08F037EC0AF0E9EC08F0E4EC08F0C4
:1002C000F7EC09F0E4EC08F0FBEC09F0E4EC08F0E2
:1002D000D8EC08F0E4EC08F037EC0AF093EC09F005
:1002E000E4EC08F0050EEF6E120001015751220DEB
:1002F000F3CF83FBF4CF84FB000E0B0183270C0E9E
:1003000084238AEC08F09DEC09F001E1000C8AECF2
:1003100008F023EC0AF0020B01E1000C8AEC08F073
:10032000100E6DEC08F0EECF80F1EDCF81F18AEC8C
:1003300008F00F0EEB5001017F6F0101100E7E6F70
:10034000F3EC09F08AEC08F037EC0AF0E9EC08F07D
:100350008AEC08F0F7EC09F08AEC08F0FBEC09F005
:100360008AEC08F0D8EC08F08AEC08F0100EC8EC23
:1003700009F0126A136A8AEC08F037EC0AF01050A0
:10038000EE261150EE221250EE221350EE2255ECC2
:100390000AF0EF9255EC0AF0EF988AEC08F022ECA4
:1003A00009F08AEC08F0EFEC09F055EC0AF0EF8266
:1003B000010C0A0E0101585D13E25851A8EC08F037
:1003C0000F0E6DEC08F0EF50FF0802E134EF14F06F
:1003D0005851A8EC08F023EC0AF0020B02E0010CE3
:1003E000000E120001015951220DF3CF81FBF4CF11
:1003F00082FB000E0B0181270C0E8223D3EC08F048
:100400009DEC09F014E1D3EC08F00F0E1BC0EBFFDC
:10041000D3EC08F0EB500201596F6CEC15F0D3EC03
:1004200008F04CEC09F0D3EC08F07BEC09F0D3ECCD
:1004300008F026EC0AF001E3000CD3EC08F0A1EC84
:1004400009F0EF885AC150F242EC14F0D3EC08F0F6
:10045000100E6DEC08F0EE2AEF22D3EC08F026EC3B
:100460000AF003E359C157F140DF010C01015B5170
:10047000220DF3CF6CFBF4CF6DFB000E0B016C274C
:100480000C0E6D23B7EC08F09DEC09F014E1B7EC0D
:1004900008F00F0E1BC0EBFFB7EC08F0EB500201A9
:1004A000596F6CEC15F0B7EC08F04CEC09F0B7ECB8
:1004B00008F07BEC09F0B7EC08F026EC0AF001E359
:1004C000000C0DEC0AF0EE24106E5F51EE20116E60
:1004D000CA0ED8801054030E11540EE2B7EC08F087
:1004E000100E6DEC08F0EECF5EF1EFCF5FF1CA0EAB
:1004F000D8805E57030E5F57B7EC08F0A1EC09F007
:10050000EF885EC153F25FC154F25CC151F25DC12C
:1005100052F264EC14F00DEC0AF0EE265F51ED227D
:10052000B7EC08F026EC0AF003E35BC157F1DDDE1F
:1005300001015E51120001016051220DF3CF00FB59
:10054000F4CF01FB000E0B0100270C0E012300CBA2
:10055000E9FF01CBEAFF52EC0AF001E1000C7AEC72
:1005600015F000CBE9FF01CBEAFFA1EC09F0EF9613
:10057000010C01016151220DF3CF20FBF4CF21FBCF
:10058000000E0B0120270C0E212318EC09F052EC71
:100590000AF02BE018EC09F023EC0AF0040B08E059
:1005A000280E1DEC09F018EC09F0A1EC09F0EF940D
:1005B00018EC09F04CEC0AF0EE50ED1008E17AEC82
:1005C00015F018EC09F0A1EC09F0EF96000C18EC0E
:1005D00009F04CEC0AF0EE06EF5AE2EC14F062C1BE
:1005E000E9FF63C1EAFFEF6E010C000C01016451E9
:1005F000220DF3CF02FBF4CF03FB000E0B01022709
:100600000C0E0323FFEC08F052EC0AF03AE0FFEC8A
:1006100008F023EC0AF0040B08E0280E1DEC09F0AA
:10062000FFEC08F0A1EC09F0EF94FFEC08F0120EDB
:10063000C8EC09F001016751105C6851115808E2DB
:10064000FFEC08F04CEC0AF0EECF67F1EDCF68F16B
:10065000FFEC08F04CEC0AF0EE50ED1008E17AECFB
:1006600015F0FFEC08F0A1EC09F0EF960AD067C195
:1006700057F268C158F265C155F266C156F220EFD3
:1006800015F0F36AF46A12000A0E0101695D07E2CF
:100690006951A8EC08F052EC0AF002E0010C000EDF
:1006A00012000B01736B6C6B0A0E6C5D01E3D4D00E
:1006B0006C51220DF3CF6DFBF4CF6EFB000E6D2756
:1006C0000C0E6E237BEC08F052EC0AF001E0C1D076
:1006D0007BEC08F023EC0AF0100B01E0BAD07BECC5
:1006E00008F0EF50000901E1B4D07BEC08F0EF50C6
:1006F000010807E17BEC08F023EC0AF0010B01E0B4
:10070000A8D07BEC08F01D0E6DEC08F00301EE5054
:10071000645D106EEE506559116E7BEC08F01F0E93
:100720006DEC08F071EC09F01050125C1150135888
:1007300001E38FD034EC14F0000901E112007BECEE
:1007400008F0F2EC08F07BEC08F01F0E6DEC08F0FE
:10075000EE2AEF227BEC08F01C0E6DEC08F0EF2A7D
:100760007BEC08F0EF50060A27E0010A25E0020AB8
:100770001CE00F0A1AE00E0A10E0060A05E0010A62
:1007800028E10B01020E24D013EC0AF0106E030EC8
:10079000105C16E20B01120E1BD00B01110E736FD1
:1007A0007BEC08F0050EEF6E14D013EC0AF0030892
:1007B00007E30B01010E0CD013EC0AF0030806E26C
:1007C0006DCB88F16ECB89F1E7DA03D00B01100E07
:1007D000736F0B01735100083CE2100E735D11E062
:1007E0007BEC08F037EC0AF0EFCF6FFBEE2AEFCF8F
:1007F00070FBEE22EFCF71FBEE22EFCF72FBEF2208
:100800000CD07BEC08F037EC0AF0EECF6FFBEECFAC
:1008100070FBEECF71FBEFCF72FBF9EC08F073CBFE
:100820007EF17BEC08F0F3EC09F06FCB76F170CB46
:1008300077F171CB78F172CB79F17BEC08F0F7ECC2
:1008400009F07BEC08F0FBEC09F07BEC08F0D8EC4D
:1008500008F00B016C2B28D71200140E0201576F01
:10086000586B02016C0E556F0B0E566F20EC15F095
:1008700001016C0E866F0B0E876F59DA6AC1E9FFB2
:100880006BC1EAFF4FEC0AF0EECF80FBEECF81FBAD
:10089000EECF82FBEFCF83FB98EC09F0EFCF84FB28
:1008A000010E6DEC08F0EFCF85FB98EC09F0020E1D
:1008B0006DEC08F0EFCF86FB98EC09F0030E6DECC1
:1008C00008F0EFCF87FB0B01886B060E896F6EC1B6
:1008D0008AFB6FC18BFB6EC1D8F26FC1D9F274EC89
:1008E00024F0F3CF8AFBF4CF8BFB0C0E0201E06FF8
:1008F000E16B0201800EDE6F0B0EDF6FA8EC24F0BF
:10090000F3CF8DFBF4CF8EFB0B018D1F8E1F240EBA
:100910001DEC09F08DCB50F242EC14F08ECB50F26E
:1009200042EC14F0140E1DEC09F06EC1E2F26FC13E
:10093000E3F204EC25F0F3CF8DFBF4CF8EFB0B013B
:100940007C51F31802E17D518E1903E07AEC15F029
:10095000010C55EC09F0106E116A140E105E000EB9
:10096000115A10C08FFB1050106E116AE85001012F
:100970006E5D6E6F11506F596F6F140E6E5F000ECB
:100980006F5B0B0155EC09F00201696F6A6B140E85
:100990006927000E6A2317EC17F06AC184F16BC156
:1009A00085F101016C0E826F0B0E836F3ED90B0136
:1009B0008C6FFE0E8C5D11E26EC18FF16FC190F1F4
:1009C00001016C0E8D6F0B0E8E6F6AC18BF16BC1C6
:1009D0008CF18CCB8AF106DA010C7AEC15F0FF0E63
:1009E0000B018C5D37E101016E510B017427010190
:1009F0006F510B017523000E762377237951020B7B
:100A000003E17951010B05E0742B000E7523762369
:100A10007723EFDB0101040E7E6F70CB7AF171CB8F
:100A20007BF172CB7CF173CB7DF174CB76F175CB1E
:100A300077F176CB78F177CB79F16CCB74F16DCB24
:100A400075F16ECB72F16FCB73F16AC170F16BC14E
:100A500071F101D8010C72C148FB73C149FB74C12B
:100A60004AFB75C14BFB76C14CFB77C14DFB78C18E
:100A70004EFB79C14FFB7AC150FB7BC151FB7CC15E
:100A800052FB7DC153FB0B015491549354955497E1
:100A90007EC155FB8DEC15F0F3CF56FBF4CF57FB21
:100AA0000B01000EF35C040EF45804E3566B040EC5
:100AB000576F0DD0360ED8805655000E575505E2AB
:100AC000360E565F000E575B02D0566B576B586B55
:100AD000596B5A6B5B6B0101480E866F0B0E876F6B
:100AE00026D9140E01018027000E81237EA30ED08B
:100AF000040E8027000E81230B01020E5C6F040E92
:100B00005D6F5E6F5F6B5499548B03D00B015489FA
:100B1000549B548D549FB8C260FBB9C261FBBAC2EA
:100B200062FBBBC263FB70C1E9FF71C1EAFF4FEC1E
:100B30000AF0EECF64FBEECF65FBEECF66FBEFCFA6
:100B400067FB686B060E696F80C16AFB81C16BFB36
:100B500080C1D8F281C1D9F274EC24F0F3CF6AFBE2
:100B6000F4CF6BFB0C0E0201E06FE16B0201600E33
:100B7000DE6F0B0EDF6FA8EC24F0F3CF58FBF4CF41
:100B800059FB0B01581F591F58CB46FB59CB47FB4C
:100B9000FF0E01017F5D02E11BC07FF1140E41DBFE
:100BA00080C157F381C158F30301060E566F70C11F
:100BB00054F371C155F3DFEC26F0140E0201536FAC
:100BC000546B0201480E516F0B0E526F64EC14F01F
:100BD00001017EA30BD0040E0201536F546B02017E
:100BE0005C0E516F0B0E526F64EC14F0140E19DB97
:100BF00080C1E2F281C1E3F204EC25F0F3CF46FBC1
:100C0000F4CF47FB240E0DDB47CB50F242EC14F03F
:100C100046CB50F242EC14F002016C6B6D6B7FC15D
:100C20006BF22AEC17F0C9EF16F00B01FE0E036F02
:100C3000026B0A0E025D4AE202511BDB84DAEF50BE
:100C4000000941E080DA0B0EA3DB50DB020E45DA2F
:100C500048DB00011250101836E11350111833E12F
:100C600072DAEF50010802E102CB03FB6CDA0D0EE1
:100C70008FDB3CDB36DB1250101825E113501118C6
:100C800022E184C1E9FF85C1EAFF4FEC0AF0EECF13
:100C900014F0EECF15F0EECF16F0EFCF17F053DAD9
:100CA000EE524FEC0AF0EE5014180DE1EE5015180C
:100CB0000AE1EE50161807E1EE50171804E103E1BF
:100CC0000B01025112000B01022BB3D70351D1DAF1
:100CD000FE0E035D27E037DAEF50010823E10A0E2C
:100CE000E66EE66A84C1E6FF85C1E6FF2CDA17DA14
:100CF0001250FCDA020E4CDB26DA0B0E10C0EBFFB2
:100D00000C0E11C0EBFFF2DA2DDA1DDAFADA1BDA7B
:100D100018DBEF9618DA63DB16DA13DBEF820B01D0
:100D200003511200FE0E035D01E1FF0CFE0CDED943
:100D3000EFCF07FBA2DBE552E750EF6ED7D92BDBF5
:100D4000020E35DB020E09DB020E2BDB020EA1DBED
:100D5000040E09DB040E30DB080E05DB080E2CDB6D
:100D60000E0E25DB0E0EF9DA0E0E1BDB0E0E91DBDE
:100D7000100E1DDB100EF1DA100E13DB100E89DBE6
:100D8000120E15DB120EE9DA120E0BDB85DB010EFB
:100D9000A4D907CBEFFF1200D1D9CFDA06E0CED924
:100DA00051DACCD91CDB84DBEF82C8D928DBC6D969
:100DB0000D0EEB6A0E0EEB6AC1D974DB02E07AEC21
:100DC00015F076DBEF96BAD91EDB72DBEF98B6D959
:100DD0003ADB010B04E0B2D9010EEF6E1200AED97E
:100DE000EF6A12000B01A26B01018A51220DF3CFB1
:100DF000A0FBF4CFA1FB000E0B01A0270C0EA1233A
:100E0000A8DAEECF98FBEECF99FBEECF9AFBEFCFAF
:100E10009BFBA6DAEECF9CFBEECF9DFBEECF9EFBBD
:100E2000EFCF9FFB6DD9040E58D948DA01018F51DD
:100E30000B019027010190510B019123000E922389
:100E4000932308DBC4DADFDAE5DA01083AE17AEC69
:100E500015F001014B2B000E4C234D234E2380DA5D
:100E600012DA0B01902B91239223932303DBF2DA06
:100E700077DA59DA69DA020B14E00A0EE66EE66AEE
:100E80008BC1E6FF8CC1E6FF2CD949D9125038D965
:100E900069D927D936DA0B01120EA26F22D9020EB8
:100EA000DCD0040EA26F90CB94FB91CB95FB92CB40
:100EB00096FB93CB97FB24D910D900DA12D99FDA8D
:100EC000D9D042DA040B04E07AEC15F088EF09F08F
:100ED00017D9080E02D99451EE1801E0C9D09551E6
:100EE000EE1801E0C5D09651EE1801E0C1D097513F
:100EF000EE1801E0BDD001E0BBD08CDA02080AE1B7
:100F0000C2DA01E1B5D0B6DA62DA040EEF6EA0D92A
:100F10002CE3AED07FDA03082AE116DA020B01E1F6
:100F2000A7D0902B000E912392239323A3DAABDA60
:100F300006E0100EA26FD5D8040EEF6E13D0120E7D
:100F4000A26FCFD8020EEF6E942B000E952396233E
:100F5000972306DA94CBEEFF95CBEEFF96CBEEFF10
:100F600097CBEEFF75D901E383D061DA83D0C8D87F
:100F7000040EB3D8EECF10F0EECF11F0B2D9E9D90C
:100F80001050EE1808E11150EE1805E11250EE185D
:100F900002E11350EE1802E07AEF15F06BDA3ADA5C
:100FA000040842E170DA09E09CD8C7D906E099D874
:100FB00049D997D814DA7FDAEF82C6D9010B15E048
:100FC0000B01110EA26FCCD9EFCF94FBEE2AEFCF1D
:100FD00095FBEE22EFCF96FBEE22EFCF97FBEF22B1
:100FE000B8D912D97ED80A0EEF6E32D941E279D83B
:100FF00059DA05E11CDA0B01100EA26F3BD00B0190
:10100000A26BAED99CCBEEFF9DCBEEFF9ECBEEFF4D
:101010009FCBEEFF9ED998CBEEFF99CBEEFF9ACBFC
:10102000EEFF9BCBEEFF24D0F5D90A0805E17AEC60
:1010300015F029DA1FE01AD0EDD9050810E17AEC95
:1010400015F082D9010B16E00B01100EA26F81D9A9
:10105000DBD819DA0BE145D8060EEF6E0BD0DAD9E2
:10106000060808E17AEC15F00EDA04E051D902D056
:101070007AEC15F00B01A25100081EE2BAD8A2CBFF
:101080007EF190CB7AF191CB7BF192CB7CF193CB3B
:101090007DF194CB76F195CB77F196CB78F197CB28
:1010A00079F12ED8DCD82CD8020E17D8DDD88BC118
:1010B00070F18CC171F1CFDC120001019151220D50
:1010C000F3CF10F0F4CF11F0000E10260C0E112209
:1010D00010C0F3FF11C0F4FF1200E926000EEA224F
:1010E0001200A0CBE9FFA1CBEAFF120086C1E9FF05
:1010F00087C1EAFF12006DCBE9FF6ECBEAFF120059
:101100008DC1E9FF8EC1EAFF12006DCBE9FF6ECB06
:10111000EAFF120083CBE9FF84CBEAFF1200EE5214
:10112000E9CF10F0EACF11F0E9CFE6FFEACFE6FF12
:10113000A8EC30F0126E060EE15E120088C1E9FFE5
:1011400089C1EAFF120000CBE9FF01CBEAFF1200E0
:10115000220DF3CFE9FFF4CFEAFF000EE9260C0ED3
:10116000EA221200EECF10F0EFCF11F012006CCB9C
:10117000E9FF6DCBEAFF1200EECF7AF1EECF7BF103
:10118000EECF7CF1EFCF7DF1120090CBEEFF91CB53
:10119000EEFF92CBEEFF93CBEEFF120001CBE9FF07
:1011A00002CBEAFF120081CBE9FF82CBEAFF1200FB
:1011B000EE52E9CF70F1EACF71F12BEF05F001CBE0
:1011C000E9FF02CBEAFF120081CBE9FF82CBEAFF05
:1011D0001200EECF76F1EECF77F1EECF78F1EFCFD0
:1011E00079F112001D0E64C3EBFF1E0E65C3EBFF09
:1011F00012000101806B816B01017F69120002CB3B
:10120000E9FF03CBEAFF1200EF2AEECF90FBEF22BB
:10121000EECF91FBEF22EECF92FBEF22EFCF93FBCD
:10122000120002016C6F6D6B7FC16BF22AEF17F039
:1012300020CBE9FF21CBEAFF12000201696F6A6B44
:1012400017EF17F00F0EEB5002015A6F72EF15F007
:101250000101000ED8808F55000E90551200EECF80
:1012600074F1EDCF75F11200EECF72F1EDCF73F1A5
:101270001200220DF3CF00FBF4CF01FB000E00277C
:101280000C0E012312004BC1EEFF4CC1EEFF4DC10D
:10129000EEFF4EC1EEFF1200100EEB6A110EEB6A6C
:1012A000280E02016C6F6D6B12007851F00BE84252
:1012B000E842E842E842040DF3501200EECF90FB02
:1012C000EECF91FBEECF92FBEFCF93FB1200EE6AD5
:1012D000EE6AEE6AEE6A1200CA0E105C030E115836
:1012E0001200EECF12F0EFCF13F0120082C1E9FF2F
:1012F00083C1EAFF12000F0EEB5002016B6F2AEF61
:1013000017F00D0E10C0EBFF0E0E11C0EBFF120018
:10131000A0CB88F1A1CB89F1CCEF06F0700EEE6E78
:10132000170EED6E1200EE2AEE22EE22EE221200D1
:101330006CC1E9FF6DC1EAFF12000F0EEB50FF0810
:101340001200210E6DEF08F0DBDE0D0EC6DEEF5051
:101350001200C7DE180E6DEF08F0BFDE3DEF0AF099
:10136000C0DE37EF0AF0B9DEEECFDAF2EECFDBF215
:10137000EECFDCF2EFCFDDF279EC24F004C010F018
:1013800005C011F006C012F007C013F076EF08F0A8
:10139000A4DEB2EF08F0010EA0DE07CBEFFF76EF80
:1013A00008F09BDEE552E750EF6E76EF08F095DE31
:1013B000EFCF07FB76EF08F090DE04C0EEFF11C020
:1013C000EEFF12C0EEFF13C0EEFF76EF08F089DEED
:1013D0001C0E83DEEF6A85DE05DF71EF08F00F0E6D
:1013E0007CDEEF681200180E78DEBCEF08F00D0E00
:1013F00074DE2FEF09F00B0E70DE34EF09F0EE52C1
:101400004ED867EF09F01F0E68DE8EEF09F07DDE23
:1014100037EF0AF066DEEF501200A9DE100E5DDE37
:1014200001015E51120067DE1C0EEB50120043D822
:10143000EF8657DE120E8FC1EBFF130E90C1EBFF4C
:101440003AD8EF8412007DDFEF501200100EA0DFBB
:101450006CEF09F085DFEECF94FBEECF95FBEECF7E
:1014600096FBEFCF97FB1200AADEA1EF09F0140E56
:101470006DEF08F06EDFC5EF08F0010E2EDEEF50C5
:10148000E66E76EF08F060DF100B120087DEA1EF4A
:1014900009F023DECBEF09F0120E6DEF08F0060E17
:1014A0006DEF08F0D0DF080B120034DEA1EF09F079
:0C14B00045DEA1EF09F015DEA1EF09F008
:0414BC000D01AA6B09
:1014C00064C3A4FD65C3A5FD0B01036B080E035D9A
:1014D00015E2500E01014F6F506B6EEC00F0E66E9E
:1014E0000B01E3DBA6EC0EF0E0DB020EC0DBEF6AE3
:1014F000DCDB090EBCDBEF6A032BE8D71200ABCDB7
:1015000000FBACCD01FB0B0100CBE9FF01CBEAFFF7
:10151000002B000E0123EF502E0807E000CBE9FF5F
:1015200001CBEAFFEF50EFE10A0C026B0251106EA3
:10153000116A100E105C000E115814E20251A0DB6B
:1015400000CBE6FF01CBE6FFF6EC30F0136E050EA4
:10155000E15E1350000903E10B01025112000B017F
:10156000022BE4D70A0CBFDB04E0200E0B01005D68
:10157000FAE00B01016B2B0E0B01005D02E1200E66
:10158000006F2F0E005D1FE05C0E005D1CE0200E62
:10159000005D1BE03F0E005D18E00D0E005D15E0E4
:1015A0000A0E005D12E00C0E015D0DE2610E005DA1
:1015B00005E300517A0802E3200E005F0151012B80
:1015C000AADB00CBEFFF8FDBD6E10B010151A3DBE0
:1015D000EF6A0B0101510CE1DF0E106E670E93DB19
:1015E000AECDE6FFAFCDE6FF0CEC31F0050EE15ECF
:1015F0003F0E0B01005D01E1010C000C0D01A45137
:101600000301645D106E65510D01A555116EE00E6C
:10161000105C2E0E115801E3AA6B0B01876B080EAC
:10162000875D06E287CBB0FD04D80B01872BF7D787
:1016300012000D01B0510A0DF3CF7CFBF4CF7DFBFE
:10164000540E0B017C270D0E7D23010E7A6F0B01CA
:101650007A5101E182D17A6B05DB64DB0AE17CDB44
:10166000EF50020B01E0AFDB77DBEF9479DBEF6A41
:101670001200F8DA020EEB50070AE9E0010A01E174
:101680005CD1030A01E12DD1010AE1E0070ADFE0A4
:10169000010A01E118D1030A01E1D6D0010AD7E11C
:1016A000E1DA4DDBD4E00B01010E7A6F64C3A4FDD7
:1016B00065C3A5FD51DBEF6A6ADB0D01B66FAAD9E0
:1016C0000B01796F49DBEF9462DB0101916F5DECF7
:1016D00008F067DBEE52060ECADA0D01A651EE18CD
:1016E00020E1A751EE181DE1A851EE181AE1A95109
:1016F000EE1817E116E1AA5102E02EDBEF84020E8C
:10170000AA5D02E0000E01D0010E106E25DB105024
:10171000010BF36EF346F346F346F70EEF14F310A6
:10172000EF6E0B01795101E089D00D016C0EAE6FA7
:101730000B0EAF6F2CDB0D01AD6F15DF0B01806F52
:10174000580E6C5D15E108DBEF50040B11E10A0E39
:10175000E66EE66AE90E106E670ED5DA6C0EE66E7E
:101760000B0EE66ED3EC30F0136E070EE15E1350F5
:101770000D016C0EAB6F0B0EAC6FC1DEE66EEADADC
:10178000E5DA0B0180510BE001016C0EE96F0B0EE5
:10179000EA6F7CCBE7F17DCBE8F1A3EC10F018DB2E
:1017A000DFDA050EEF6EE6DAD1DA00DB106E060E38
:1017B000105C30E312DB04082DE36C0EE66E0B0EBA
:1017C000E66E25EC31F0E552E552F3CF7BFB05DB0D
:1017D000030802E3030E01D0020E0B017B5FFDDA6A
:1017E0000B0FE66EB7DAB2DAF8DA4ADA7B51146A2E
:1017F0006C0F136E0B0E142213C0E6FF14C0E6FF2D
:101800000CEC31F0156E050EE15E1550B3DAE552C1
:10181000E750EF6ECBDAFF0803E1D3DAEF6A06D0C8
:10182000C5DAFE0806E1CDDA030EEF6E99DA050E91
:1018300082D092DAEF8294DA010E7DD0790501E050
:1018400006D78EDA030E77D0B5DA01E100D70B01A7
:10185000010E7A6F0D01680EBB6F670EBC6F4EDA1A
:101860000D01780EBB6F670EBC6FA7DA73DAEF3429
:10187000EA6AFE0BEA36E96E6E0EE926020EEA22ED
:10188000EECFBBFDEDCFBCFD39DA64DAEFCF10F05F
:101890000B0E105C06E30D01870EBB6F670EBC6F6D
:1018A0008CDAB0CDB9FDA6D998DA060803E154DA8E
:1018B000EF8002D051DAEF90D5D9030ED8D9EF6A74
:1018C0004FDA020E38D0CED93ADA01E081DA7CCB99
:1018D000B7FD7DCBB8FDDCD8000901E1B8D673DADD
:1018E00028D068DA01E1B3D66CDAEF34EA6AFE0B8D
:1018F000EA36E96E8E0EE926020EEA22EECF7EFB74
:10190000EDCF7FFB0B017ECBF6FF7FCBF7FF7E2B6E
:10191000000E7F230800F5CF7BFBF55005E07BCB65
:101920005AF1A0D9D1D9EED732DA0101576F75EC4F
:1019300001F016DA060EEF6E8AD694D9F3D90AE0D2
:1019400039DA08E024DA0101566F35EC01F008DAE3
:10195000070EEF6E01DAEF947AD61200B4CDE9FFEC
:10196000B5CDEAFFEF040B011E6F1D6BEF6A1F6B15
:101970001E510D01EA6AB225E96EB351EA22EF6AFF
:101980000B011F5141E101011C0E626F0B0E636FD1
:10199000B1CD61F1B9EC02F0000936E03D0E0B016A
:1019A0001C5D0BE11C6B1E511D5D1EE21D29B4CD9B
:1019B000E9FFB5CDEAFFEF6E17D0260E1C5D02E100
:1019C000020E0AD0200E1C5D06E00D0E1C5D03E029
:1019D0000A0E1C5D04E1010E1F6F1C6B05D02B0E5F
:1019E0001C5D02E1200E1C6F1E511D5D06E2B2CD92
:1019F000E9FFB3CDEAFF1CCBEFFF0D01B22B000EC8
:101A0000B3230B011D2BBCD70B011F5101E1000CAF
:101A10001F0512000B01056B040E055D19E205514F
:101A20000101626F636B000E62270B0E6323B6CD5C
:101A300061F1B9EC02F000090BE00B010551052B37
:101A4000EA6A000FE96E0B0EEA22EF502008E4E18B
:101A50000B010551EA6A000FE96E0B0EEA22EF6AEC
:101A6000470E005D07E1450E015D04E1540E025D85
:101A700001E1000C500E005D0AE14F0E015D07E12F
:101A8000530E025D04E1540E035D01E1010C020CF2
:101A9000F2D813D901E1A6D00B01856BECD8030E67
:101AA000EB50040818E0E7D814D9400B0DE1E3D857
:101AB000010EEB500201386F8FEC23F00B01866FA3
:101AC000DAD807D9200B07E0D6D8EF500101576FBD
:101AD00075EC01F0010CCFD8090EC9D8EF50010BFD
:101AE00001E17BD0C8D8030EEB50040A50E0070A8E
:101AF00034E0010A1BE0030A0BE0010A6BE1250E4A
:101B0000865D03E131D9010E26D0010E856F62D0CA
:101B1000250E865D03E1010E856F5AD029D9030E8B
:101B2000A6D886CBEFFF20D9020E15D0610E865DB8
:101B300002E3270E04D0410E865D02E3070E865FA6
:101B4000300E865D100DF350E66E12D9020E8FD85E
:101B5000FDD80AD9030EEF6E3DD0610E865D02E31B
:101B6000270E04D0410E865D02E3070E865F300E1D
:101B7000865D106EFDD8020E7AD81050EF12F4D8A0
:101B8000040EEF6E78D873D8EE6AED6A23D00101A7
:101B9000860EED6F0B0EEE6FB7CDEBF1B8CDECF11D
:101BA00040EC11F0F3CF10F0F4CF11F0E1D8F3CF07
:101BB000EEFF11C0EDFF0B01010E856FD9D8FF0EAE
:101BC000EE1808E1FF0EED1805E1865101E1856B85
:101BD000CBD8EF6A855101E15BD786CB5AF14BD860
:101BE00073D856D748D8010EEB500201376F68EC16
:101BF00023F0000C0D01B9510A0DF3CF85FBF4CF92
:101C000086FB540E0B0185270D0E862301010D0E58
:101C1000C1D801010A0ECAEF0EF00D01BA510A0D2A
:101C2000F3CF85FBF4CF86FB540E0B0185270D0EF9
:101C30008623BBCDF6FFBCCDF7FF0800F55011E0C1
:101C40000D01BBCDF6FFBCCDF7FFBB2B000EBC23B7
:101C50000800F5CF5AF185CBE9FF86CBEAFF34D8EF
:101C6000E8D712007CCBE9FF7DCBEAFF1200E92622
:101C7000000EEA221200B7CDE9FFB8CDEAFF12004C
:101C8000040DF3CFF6FFF4CFF7FF280EF626670E0C
:101C9000F722F6CF10F0F7CF11F0126A10C0E6FF6E
:101CA00011C0E6FF12C0E6FF120003510A0D79D8F9
:101CB000540EE9260D0EEA221200EF500101586F72
:101CC000D9EC01F000091200EF500101596FF2EF59
:101CD00001F0010EEB50080D64D8000EE926020E4B
:101CE000EA22EF5012000101000E626F0B0E636FCB
:101CF000ADCD61F1B9EC02F0000912005ED8B0CDB3
:101D0000B9FDFAEF0DF0116E126A10C0E6FFE66E33
:101D100012C0E6FF12000D01EA6AAE25E96EAF516E
:101D2000EA221200EF500101556F2CEC01F000097E
:101D30001200010EEB500201366F60EF23F0EF50FE
:101D40000101696F44EC03F000091200E552E7500D
:101D5000EF6E120036D844D085DF090E37EF0EF053
:101D600081DF020E37EF0EF086DF030E37EF0EF045
:101D700082DF36D00201356B02016C0E336F0B0E21
:101D8000346FC3EC22F0E66E6DDFEE5212006ADFB4
:101D9000EF5012005A6F85CBE9FF86CBEAFF64EF64
:101DA0000EF0F3CFE9FFF4CFEAFF12005BDF010E84
:101DB000EB50120057DF5DEF0EF0B0CDBAFD0DEF26
:101DC0000EF050DF0DD0C8DFEF924CDF99EF0EF030
:101DD000DEDF0101606F9BEF02F0BCDFEF5012000D
:061DE000040E37EF0EF0C7
:0A1DE600120053EC13F0040B06E0AA
:101DF00053EC13F0080B01E0020C010C000C0B017A
:101E00001C6B1D6BE2C1E9FFE3C1EAFFEF506B08F9
:101E100001E080D00B01010E206F0201210EE76F5F
:101E20000B0EE86F010E0101E2250201E56F000EC5
:101E30000101E3210201E66F7EEC25F0000903E1D8
:101E4000F36AF46A7FD1E4C1E6FFE5C1E6FF5EEC28
:101E50002BF0E552E552F3CF22FB0B012151110883
:101E600004E2160E0B01215D05E10B011C830B0141
:101E7000206B43D00B012151150809E3130E0B0110
:101E8000215D04E00B011C8F0B01206B36D00B0190
:101E900021511A0801E331D00B0121511E0801E341
:101EA0002CD00B012151220817E31F0E0B01215DDD
:101EB00004E0210E0B01215D07E10B01225108080E
:101EC00002E30B01206B02D00B01206B0B012051B0
:101ED00002E10B011C8511D00B012151300805E3F3
:101EE0000B011C870B01206B08D00B01215132081C
:101EF00004E30B011C890B01206B0B01205109E14C
:101F00000101E65106E022CBA8FF21CBD7F29EECDF
:101F100031F013D1E2C1E9FFE3C1EAFFEFCF10F0E6
:101F2000610E105C01E2B5D0E2C1E9FFE3C1EAFF56
:101F3000EF50670801E2ADD0E2C1E9FFE3C1EAFF7B
:101F4000EF50640807E0E2C1E9FFE3C1EAFFEF50A8
:101F5000650803E1F36AF46AF5D0E2C1E9FFE3C181
:101F6000EAFFEF509F0F0B011E6F1F6B890E0B01D5
:101F70001E270F0E0B011F23010E0101EA6AE22545
:101F8000E96EE351EA22EF5014E10201200EE76FFF
:101F90000B0EE86FE4C1E5F2E5C1E6F27EEC25F058
:101FA000000906E01ECBE9FF1FCBEAFF20CBEFFFC5
:101FB0006FD0010E0101EA6AE225E96EE351EA22DF
:101FC000EF50780833E1020E0101EA6AE225E96E7A
:101FD000E351EA22EF50D00F106E010E105204E0D0
:101FE000E846FE0B1006FCE10B01206FE4C1E9FF9F
:101FF000E5C1EAFFEF5031080AE10B01201D106E28
:102000001ECBE9FF1FCBEAFF1050EF160ED0E4C144
:10201000E9FFE5C1EAFFEF50300807E11ECBE9FF19
:102020001FCBEAFF0B012051EF1232D0010E01014C
:10203000EA6AE225E96EE351EA22EF50D00F106E12
:10204000010E105204E0E846FE0B1006FCE10B0105
:10205000206FE4C1E9FFE5C1EAFFEF5030080AE173
:102060000B01201D106E1ECBE9FF1FCBEAFF1050A5
:10207000EF160ED0E4C1E9FFE5C1EAFFEF503108E9
:1020800007E11ECBE9FF1FCBEAFF0B012051EF1246
:1020900054D0E2C1E9FFE3C1EAFFEF506C082DE143
:1020A0000101E65129E0010E0101EA6AE225E96E2B
:1020B000E351EA22EF50610A11E0030A01E01CD06B
:1020C0000201080EED6FE4C1EBF2E5C1ECF23E0E49
:1020D0000201E96FEA6BA3EC25F00ED00201080EB5
:1020E000ED6FE4C1EBF2E5C1ECF2350E0201E96FF0
:1020F000EA6BA3EC25F000D020D0E2C1E9FFE3C1F8
:10210000EAFFEF506D0819E10101E65116E0E4C164
:10211000E9FFE5C1EAFFEF50720A01E00ED0D3EC0F
:1021200016F0FF0E986E966E956E936E000E866E8C
:10213000846E836E816EFF0000D01CCBF3FF1DCB3D
:10214000F4FF00D012000B01146B156B186BE7C184
:10215000E0F1E8C1E1F148DE0B01196F140E166FD2
:102160000D01160EB46F0B0EB56F0D01000EB26FA0
:102170000B0EB36FB1DAEF500D01B16FAEEC0CF096
:102180000B01176F182B1B6B6C0E005D36E10151B4
:10219000750A2BE0050A45E1010E1B6F3E0E54DA6D
:1021A00040E1020E0B01185D3CE1010E1A1539E009
:1021B00093DAEF500101916F5DEC08F0F3CFE9FF86
:1021C000F4CFEAFFEE52060E83DAEECFA6FDEECF95
:1021D000A7FDEECFA8FDEFCFA9FD0D01010EAA6F5F
:1021E00043DAEF8441DAEF961CD0010E1B6F350EF7
:1021F0002BDA17E10B011A8114D06D0E005D11E18D
:1022000019510FE01651EA6A000FE96E0B0EEA222F
:10221000EF506F0A06E1010E1B6F0D01AA6B24DA65
:10222000EF940B011B5115E119CBE6F11651010199
:10223000E46FE56B000EE4270B0EE5230101000EB1
:10224000E26F0B0EE36FDBDDF3500B011413F45060
:102250001513175101E082D71451020B01E012004F
:102260001451040B02E0B2EF31F01451080B02E0FC
:1022700001EF32F01451100B02E02DEC32F012009D
:10228000F7D9020E25DAEFCF01FBF2D9030E20DADF
:10229000EFCF02FBEDD9EECF07FBEDCF08FB13DA52
:1022A000EF6AEBC1E0F1ECC1E1F19EDD0B01096FDA
:1022B000610E025D6DE3025168086AE3006B610E16
:1022C000025D066F070E0115106E010E105204E03C
:1022D000E846FE0B1006FCE10B01056F0651036F8B
:1022E000046B920E03270F0E0423D0D909E1065187
:1022F000036F046B890E03270F0E0423008107D0A0
:102300000651036F046B800E03270F0E0423F00E9B
:102310000115066FE85004E1B9D934E0310E35D02B
:10232000100E065D0CE1B2D905E10101C80EF26F95
:10233000680E02D10101C50EF26F680EFDD0200EAD
:10234000065D03E1010E001506E0300E065D08E1B2
:10235000010E001505E0080E011501E1D8D0E8D006
:10236000400E065D08E1010E001505E00101AB0E0F
:10237000F26F680EE1D0500E065D01E0E6D0010E6E
:10238000001502E0300E01D0310E9DD9EF6EDDD088
:102390006B0E025D0AE1095101E1D7D001CBD6F203
:1023A00094EC31F00101FC6F62D06C0E025D42E1F1
:1023B00009512CE00151040A24E0060A1DE0030A39
:1023C00016E0010A01E0C1D009050CE1350E01015A
:1023D000F76FF86BEDC1F5F1EEC1F6F107CBF4F153
:1023E000C7EF12F00101250EF26F500EA5D00101CA
:1023F000D00EF26F690EA0D00101D60EF26F690EF9
:102400009BD00101220EF26F500E96D00151030AAB
:1024100008E0030A01E099D001011C0EF26F500E92
:102420008BD0095102E1300E01D0310E066FE8CF9A
:10243000FCF11DD06E0E025D01E087D0006B0F0E27
:102440000115106EC11C0F0B105C01E20083F00E31
:102450000115066FE85005E10101920EF26F680E5A
:102460006BD0100E065D0BE126D9EFCFFCF1EDC16C
:10247000FAF1EEC1FBF107CBF9F1E8EF12F0200E13
:10248000065D39E118D9EFCF06FB0751081120E1AD
:10249000330E03D90750300F0101DA6F2E0EDB6FB8
:1024A000330EFBD803C006FB0B0103500A0DB8D84E
:1024B0000101DC6F0A0EF1D807C006FB0B010750C3
:1024C000640DAED80101DD6FDE6B0B01076B086B8D
:1024D0000751D5D8F8D8EF6E0751D1D836E007CBE1
:1024E00010F008CB11F0072B000E082307CBF3FFE9
:1024F00008CBF4FF1200300E065D03E1020E00155A
:1025000006E1500E065D08E1020E001505E101012D
:10251000BC0EF26F680E10D0400E065D03E1020E95
:10252000001506E1600E065D10E1020E00150DE1DA
:102530000101C10EF26F680EF36FEDC1F0F1EEC153
:10254000F1F107CBEFF1A8EF12F0F368F468120095
:102550000101EF51F76AF225F66EF351F7220800F8
:10256000F550F0C1E9FFF1C1EAFFEF6EF0C1E9FFFC
:10257000F1C1EAFFEF5003E1F368F4681200EF2BBA
:10258000EF51116AEFC1F3FF11C0F4FF1200010116
:10259000F451F7250B010A6F000E0101F821AA6E14
:1025A0000ACBA9FF3F0EA616A680A850F5C1E9FFE9
:1025B000F6C1EAFFEF6EA85003E1F368F468120079
:1025C000F42BF451116AF4C1F3FF11C0F4FF1200AF
:1025D0000101F95110E1DA0EE66E010EE66EFC51D2
:1025E000E66EE66AD3EC2BF0E552E552E552E55291
:1025F0000101DF6BF96BF95142D8FAC1E9FFFBC168
:10260000EAFFEF6EF9513BD803E1F368F46812007A
:10261000F92BF951116AF9C1F3FF11C0F4FF12004F
:10262000F3CF10F0F4CF11F0330E0B6E0C6AF3CF32
:1026300006F0F4CF07F09CEC34F006C010F007C0B1
:1026400011F0300E062412000201F06FF16B0B0145
:1026500016510201EE6FEF6B000EEE270B0EEF230B
:10266000DBEC25F00009120037D8090E68EF13F0F3
:10267000EBC1E9FFECC1EAFF040E68EF13F0EA6A70
:10268000DA0FE96E010EEA22EF50120003CBE9FFE8
:1026900004CBEAFFEF5005151200106E0C6E06CB4E
:1026A00007F0C3EF34F0E0C1E9FFE1C1EAFF090E32
:1026B0000FD8EF5012000F0E0115EA6ACA0FE96E2B
:1026C000020EEA221200EDC1E9FFEEC1EAFF12009C
:1026D000E926000EEA221200E7C1E9FFE8C1EAFF9D
:0226E0001200E6
:0E26E200966A8688988802014A6B4B6B4C6B97
:1026F0004D6B4E6B4F6B0B01006B0051106E116AEE
:10270000D890115004E6010E105C000E115814E22E
:102710000051040DF3CF10F0F4CF11F0400E10264D
:10272000000E11220051AFDB10C0EFFF0051ABDBF8
:10273000EE52EF80002BE1D71B6A0201496933DBBF
:10274000B7DB02011F0EB1DB0201656F02011F0E34
:10275000A9DBAEDB0201210EA0DBAADB0201080E21
:10276000656F02010E0EC7DB0A0EC5DB0B0ED1DB57
:10277000040E656F02010C0ECCDB020E656F0201C8
:102780000D0E90DBDBDB8EDBB1DB010EC2DB600EFE
:10279000656F0201020E86DBA9DB030EBADB6569F9
:1027A0000201070EA8DB0F0EB4DB610E76DBBCC2A4
:1027B00065F20201010E76DBBDC265F20201020E76
:1027C00071DBBEC265F20201030E6CDBBFC265F2B3
:1027D0000201040E67DBC0C265F20201050E62DB76
:1027E000C1C265F20201060E5DDB0B01006B080E33
:1027F000005D0AE202016569080E0B010025020175
:1028000051DB0B01002BF3D771DB070E4BDB440EC2
:10281000186E0201220E41DB51DB0D0E7ADBE00E59
:102820003CDB0201C00E656F0201010E64DB040E89
:1028300062DB010E6EDB200E4DEF17F002010D0E74
:1028400070DB02014A2711504B2302010E0E69DB97
:1028500002014C2711504D2302010F0E62DB0201D1
:102860004E2711504F231200020149511B5C09E110
:102870000201666BB3DA040B03E10201496964D318
:10288000000C62D325DB86A8FED78D8C6B0E8D6E77
:10289000836A8D9C86A8FED722DB86A8FED78D8C06
:1028A000670E8D6E400E836E8D9C86A8FED78D8C34
:1028B000700E8D6E50C283FF8D9C86A8FED78D8CC6
:1028C000192A000E1A22120002015351541101E17B
:1028D0001200010E5315106E116A535110240B0192
:1028E0003E6F0201545111200B013F6F956A670E34
:1028F0008D6E400E836E8D9C86A8FED78D8C6A0EE1
:102900008D6E3ECB83FF8D9C86A8FED78D8C6B0E83
:102910008D6E3FCB83FF8D9C86A8FED7E0DA86A81C
:10292000FED78D8C02015351192654511A22700E74
:102930008D6EE4DA86A8FED78D8C53C23CFB54C260
:102940003DFB0B01010E3C5F000E3D5B0B013CCBE0
:1029500010F03DCB11F03C07000E3D5B1050111004
:1029600030E0080E3C5D000E3D5926E389DA86A86A
:10297000FED78D8C85DA86A8FED78D8C81DA86A865
:10298000FED78D8C7DDA86A8FED78D8C79DA86A865
:10299000FED78D8C75DA86A8FED78D8C71DA86A865
:1029A000FED78D8C6DDA86A8FED78D8C080E0B01B4
:1029B0003C5F000E3D5BD5D763DA86A8FED78D8CD1
:1029C000C5D7120085DA86A8FED78D8C6B0E8D6E6A
:1029D000836A8D9C86A8FED78D8CFF0E195C1DE145
:1029E0005F0E1A5C1AE10B013269336932CB67F270
:1029F00033CB68F201DA66DA86A8FED78D8C020145
:102A0000100E53DA0B01316F326B440E336F32CB41
:102A100067F2E8CF68F2F0D910D054DA86A8FED772
:102A20008D8C9568700E8D6E8D9A86A8FED783CF9B
:102A300031FB8D8A192A000E1A220B013151120026
:102A400057C2B5FB58C2B6FB02015751581103E1FA
:102A5000F36AF46A1200956A6A0E8D6EB5CB83FF35
:102A60008D9C86A8FED78D8C6B0E8D6EB6CB83FFAA
:102A70008D9C86A8FED78D8C25DA86A8FED78D8CF6
:102A80000B01B5511926B6511A22600E1A5C02E3E9
:102A90001C0E1A5E9568700E8D6E0B01B5CB10F092
:102AA000B6CB11F0B507000EB65B105011100FE059
:102AB0008D9A86A8FED7020155C2E9FF56C2EAFFE9
:102AC000552B000E562383CFEFFF8D8AE6D757C2D2
:102AD000F3FF58C2F4FF120002015951D4D9EE524B
:102AE000EF90120002015A51CED9EE52EF805AC235
:102AF0001BF0120018C036FB0B01010E356FE8CF3A
:102B000067F218C068F278D95DDF0B01346FE8CF47
:102B100065F20201030E52EF17F0FED90B01006FB0
:102B20000201200EBAD918500B01005D05E2600EBB
:102B3000D8801854002502D01850005D016FE8506D
:102B4000106E116A1C0ED8801056000E115610C05F
:102B500001FB10C003FB026B02CBF3FF10C0F4FFBC
:102B600012000201E00EE5D90B01006F0201200EF8
:102B700094D90B010051040B01E0000C010C5DC263
:102B8000E9FF5EC2EAFFEF68C7D90B01126F0201CD
:102B9000200ECFD90B01136FDCD9100B37E00201E7
:102BA000666B1CD9040B0B01176F0201210E75D93E
:102BB000020EE66E85EC34F0E55280D90A0E9BD900
:102BC0000B0E70D90B01175108E0C3D90A0B02E0B4
:102BD000000E01D0010E0B01176F0201020E656F8E
:102BE00002010D0E96D9220E58D912CB18F082DFB1
:102BF000020165690201070E7ED90D0E53D90B0142
:102C0000175103E00201260E48D9000C0B011351A5
:102C1000125D67E013CB15FB146B14CB67F213CB7B
:102C200068F2EAD8120E0201576F586B0201000ECB
:102C3000556F0B0E566F04DF0B010051010B4EE078
:102C4000400E025D000E035949E3EE0ED880025596
:102C5000050E035543E3600E015D40E20151106E25
:102C6000116AD890115004E6440E105C000E115801
:102C700035E310CBD8F211CBD9F274EC24F0F3CFBA
:102C800010FBF4CF11FB060EE66EE66A0A0EE66E46
:102C90000B0EE66E5BC2E9FF5CC2EAFF5BC210F09E
:102CA0005CC211F05BC2E6FF5CC2E6FFA8EC30F04C
:102CB000126E060EE15E1250080E0B01115D0BE163
:102CC000105103E0060E105D06E15DC2E9FF5EC231
:102CD000EAFF10CBEFFF13CB18F0010C12CB18F06A
:102CE00009DF000C02010A0E656F0201070EDAD837
:102CF0001DD9EFCF41FB0B01406B40CB67F241CBBD
:102D000068F27AD8060E0201536F546B5FC251F21B
:102D100060C252F2D9DDBCC250F2B4DDBDC250F285
:102D2000B1DDBEC250F2AEDDBFC250F2ABDDC0C2FB
:102D300050F2A8DDC1C250F2A5DD0201615103E1EC
:102D40000B01426B03D00B01060E426F0201080E0D
:102D5000506F98DD42CB50F295DD0E0E02016227D6
:102D6000000E63233C0E625D000E635903E23C0ECD
:102D7000626F636B62C240FB63C241FB62C265F279
:102D80000201050E8FD841CB65F20201060E52EF0B
:102D900017F0D4D8BED8240E80D81BC049F2C6D8AC
:102DA000EE52EF8012009568600E8D6E8D8C8D8ACC
:102DB0008D8E966A0A0EE66EDDEC34F0E55278D818
:102DC0008D9E1200600E020164118D6E65C283FF3C
:102DD000956A8D9C86A8FED78D8C12009568600E32
:102DE000020166118D6E8D9A86A8FED783CF37FBC0
:102DF0008D8A0B013751120067C219F068C21AF0B0
:102E000067C265F20201080E4DD868C265F2020180
:102E1000090E52EF17F00201090E47D80B01016F9E
:102E20000201080E42D8F36E01CBF4FF120018C065
:102E300023FB0B01120E226F020169510B012227A5
:102E400002016A510B01232322CB67F223CB68F2E4
:102E5000FCEF16F06BC21BF069D8EFCF0DFB0B0136
:102E60000E0E0C6F02016C510B010C2702016D510B
:102E70000B010D230CCB67F20DCB68F2FCEF16F0C3
:102E800002017EEF17F0E96EEA6AD890E936EA3679
:102E9000460EE926020EEA221200656F0201646BFB
:102EA000E2EF16F0646FE2EF16F0666FEEEF16F0E9
:102EB000050EE66E85EC34F0E55212000201656BFA
:102EC00002011200600E8D6E0A0E836E8D9C120040
:102ED000956A6A0E8D6E010E836E8D9C12008D8C2C
:102EE000600E8D6E120E836E8D9C12000201440ED8
:102EF000656F02011200D6DF5EEF17F051C2E9FFE5
:102F000052C2EAFF512B000E5223EF50836E8D9C6C
:102F10001200C8DF020112000201600EBEDFA9EF3D
:102F200017F0C3DF106E116AE85012001B5043EF18
:102F300017F0B3DF0201030E55EF17F0F7DFEFCF05
:102F400065F20201040E1200F1DFEE52EF50010BA8
:0A2F500012000201070E55EF17F002
:062F5A000B01006B020EEA
:102F6000005D07E200513BDB00512DDBEF90002BB1
:102F7000F6D712000B01000E016F010E026F006BFD
:102F8000020E005D43E2DCDA0C0EC7DACADA126A1E
:102F9000136A105011101210131032E1D1DA0C0E16
:102FA00029C1EBFF0D0E2AC1EBFF01012B512C11A2
:102FB00011E00A0EE66EE66A2BC1E6FF2CC1E6FFC1
:102FC000BFDA01CB10F002CB11F001CBE6FF02CB50
:102FD000E6FFD8DAB5DA0A0E2DC1EBFF0B0E2EC1D3
:102FE000EBFFAEDA0E0EEB6A0F0EEB6AA9DA100EEB
:102FF000EB6A110EEB6A00CB28F10B0100511200B5
:10300000140E0127000E0223002BBAD7FF0C01017A
:103010002F51EFEF1AF0020E0101305D04E230C1D2
:1030200028F134EF14F0000C01012851140DF3CFF6
:103030000AFBF4CF0BFB000E0B010A27010E0B233A
:10304000CADAEE50ED1004E190DA94DA8EDA87DA1B
:1030500031C150F242EC14F0BEDAEE2AEF22BBDAB4
:10306000C4DA01E346D8010C01012851140DF3CF55
:103070000AFBF4CF0BFB000E0B010A27010E0B23FA
:10308000A6DAEE50ED1004E151DA74DA4FDA67DABD
:103090009EDA01013451EE24106E3551EE20116E8E
:1030A000D60ED8801054030E11540AE290DAEECFF7
:1030B00034F1EFCF35F1D60ED8803457030E3557A3
:1030C00034C153F235C154F232C151F233C152F21C
:1030D00064EC14F07CDA01013451EE263551ED2216
:1030E00076DA83DA01E305D834C1F3FF35C1F4FFA2
:1030F000120001012851140DF3CF08FBF4CF09FB96
:10310000000E0B010827010E092315DA0C0E05DA53
:1031100040DAF3CF00FBF4CF01FB0DDA0A0EFDD944
:1031200038DAF3CF02FBF4CF03FB05DA0E0EF5D944
:10313000EECF04FBEFCF05FB080E0B010427000EBA
:103140000523066B076B140E02016C6F6D6BF3D9D0
:1031500006DA04CB57F305CB58F30301110E566F73
:10316000EAD908CB54F309CB55F3DFEC26F004CBB6
:10317000D8F205CBD9F274EC24F0F3CF04FBF4CFF2
:1031800005FB080E0201536F546B0201000E516FD4
:103190000B0E526F64EC14F0C9EC16F0CCD9120E81
:1031A000BCD9EF68C8D90E0EEB6A0F0EEB6A12009D
:1031B000020E0101365D0AE236C128F1FFD9D8803E
:1031C000EE54000EED5401E3000C010C000C17DA74
:1031D00001E1000C2851F7D9EF50010B01E013DA9F
:1031E000E2EC14F037C1E9FF38C1EAFFEF6E11DA03
:1031F000EE06EF5AE3D9EE50ED1002E17AEC15F04D
:10320000010CFDD903E1F36AF46A12002851DBD9FD
:10321000EF50010B01E0F7D9FCD983D93B51105C89
:103220003C51115805E2CAD9EECF3BF1EDCF3CF14C
:103230003BC157F23CC158F239C155F23AC156F27E
:1032400020EC15F0F3CF00FBF4CF01FBE2D90B012A
:103250000051EE5E0151ED5AD2D902E17AEC15F03F
:103260003BC1F3FF3CC1F4FF1200C9D902E07AEC84
:1032700015F0CFD9EE6AED6A1200080E0201576F01
:10328000586B0201460E556F0B0E566F20EC15F071
:1032900046CB5DFB47CB46FB5DCB47FB48CB5DFB9D
:1032A00049CB48FB5DCB49FB080E106E0B014B511F
:1032B000D880105403E24A055D6F02D04ACB5DFB13
:1032C000080E4B5D4A6F5DCB4BFB4CCB5DFB4DCB92
:1032D0004CFB5DCB4DFB3DC1E9FF3EC1EAFF060E55
:1032E0001CD9EECF4FFBEECF50FBEECF51FBEFCF13
:1032F00052FB55D9EFCF53FB010E0FD9EFCF54FB43
:103300004ED9020E0AD9EFCF55FB49D9030E05D984
:10331000EFCF56FB576B110E586F41C159FB42C19D
:103320005AFB41C1D8F242C1D9F274EC24F0F3CF78
:1033300059FBF4CF5AFB0C0E0201E06FE16B020166
:103340004F0EDE6F0B0EDF6FA8EC24F0F3CF5BFBAC
:10335000F4CF5CFB0B015B1F5C1F1A0EFBD85BCB31
:1033600050F242EC14F05CCB50F242EC14F0140E2C
:10337000F1D841C1E2F242C1E3F204EC25F0F3CF0F
:103380005BFBF4CF5CFB0B014C51F31816E14D5184
:103390005C1913E13FC147F140C148F13DC145F11E
:1033A0003EC146F10101460E436F0B0E446F1CD81F
:1033B0000B014E6FFF0E4E5D03E17AEC15F0010C30
:1033C0004E51A1D8100EA9D84ACBEEFF4BCBEDFF42
:1033D0004E51F9D8EF80010C0101285194D8E9CF62
:1033E000F3FFEACFF4FF12000B010169000E026F38
:1033F000010E036F006B020E005D5BE2A6D80C0E9F
:10340000FAD8020E8AD8D5D80001125010184AE115
:103410001350111847E199D80A0EEDD8CAD81250A6
:1034200010183EE1135011183BE18FD8100E75D8DB
:10343000EECF14F0EFCF15F0166A176A145015107E
:10344000161017102DE145C1E9FF46C1EAFF060E2F
:1034500064D8EECF10F0EECF11F0ABD876D8060ED0
:103460005CD8EE50101808E1EE50111805E1EE504E
:10347000121802E1EE50131810E047C1E9FF48C1ED
:10348000EAFFE868EE180CE1E868EE1809E1E86880
:10349000EE1806E1E868EE1803E10B010051120096
:1034A00000CB01FB0B01140E0227000E0323002B9F
:1034B000A2D7FF0E015D24E00151140DF3CF02FBF2
:1034C000F4CF03FB000E0227010E03230A0EE66E63
:1034D000E66A45C1E6FF46C1E6FF37D802CB10F0E9
:1034E00003CB11F002CBE6FF03CBE6FF4BD85CD851
:1034F00018D82BD80A0E10C0EBFF0B0E11C0EBFF33
:103500000B0101511200140DF3CFE9FFF4CFEAFFD4
:10351000000EE926010EEA221200E926000EEA2238
:103520001200EECF10F0EFCF11F012000ACBE9FF3E
:103530000BCBEAFF120008CBE9FF09CBEAFF120030
:1035400001CBE9FF02CBEAFF120002CBE9FF03CB7C
:10355000EAFF12000201696F6A6B17EF17F0120E93
:10356000EB5002016B6F2AEF17F00ACBE9FF0BCB90
:10357000EAFF1200120E1BC0EBFF1C0E02016C6F63
:103580006D6B1200A8EC30F0126E060EE15E125068
:103590001200EECFD8F2EDCFD9F274EF24F03FC194
:1035A000E9FF40C1EAFF120043C1E9FF44C1EAFF5D
:1035B0001200EECF12F0EFCF13F012002851A3DF6C
:1035C000100E8DEF1AF09FDF130E8DEF1AF0AEDFA5
:1035D0000E0E8DEF1AF0C9DF0E0E8DEF1AF093DF8D
:1035E0000C0E9BDFEE6AED6A12009BDFD60E105CBC
:1035F000030E1158120091DF94DFD4EF1AF009D8AE
:10360000EE50ED1012002851DEDFEF901C0EAAEFF5
:083610001AF00101DEEF1AF0CF
:08361800070E0301755D01E1DD
:103620001200FF0E765D01E0A7DA03017669756B83
:10363000786B120003017551060A01E1A2D0030A5A
:1036400066E0010A59E0070A46E0010A33E0030A8E
:1036500027E0010A01E012000B010E690F691069F1
:1036600011691269136914691569166917690301EB
:10367000086B096B0A6B0B6B430E01012D6F2E6BF0
:1036800001010E0E2B6F0B0E2C6F440E0101296FE2
:103690002A6BBAEC17F00301766F62DA010E756FD0
:1036A00050DA140E105C000E115801E27DD00301B7
:1036B000020E3BD00301085109110A110B1133E12D
:1036C00076C330F10BEC18F000096EE00301010E37
:1036D0005FDA030E2AD061DA03E30301020E756F8D
:1036E00076C336F1D8EC18F000095EE063D8020822
:1036F0005BE10301040E756F76C330F10BEC18F03B
:10370000000952E00301030E43DA050E0ED076C322
:1037100036F1D8EC18F000092EE04CD80B01186FE8
:10372000060E185D04E10301040E756F1200050E0C
:10373000185D26E121DA0301766912DA060E756F4B
:1037400008C3B8F209C3B9F20AC3BAF20BC3BBF299
:1037500010C3C2F211C3C3F212C3C4F213C3C5F241
:103760000CC3C6F20DC3C7F20EC3C8F20FC3C9F231
:103770007781782B120011DA17E30301020E756FBF
:103780001200DFD9640E105C000E11580DE304071F
:10379000000E055B065B075B04510511061107115E
:1037A00002E10301756BDCD912000301080E756F8D
:1037B000BCEF1DF00B01026B03013C0E046F056BA7
:1037C000066B076BB0D9020E0B01005D01E0EBD078
:1037D000016B0F0E015D02E2EFD9FBD70101080E6C
:1037E000376F030EABD9090E376F030EA7D90A0E38
:1037F000376F030EA3D90B0E376F030EC6D90B011B
:10380000016B080E015D02E2D7D9FBD7BCC208FBF1
:10381000BDC209FBBEC20AFBBFC20BFBC0C20CFB90
:10382000C1C20DFB016B060E015D0EE27CD90B01DE
:103830000151EA6A080FE96E0B0EEA22EF50005DB3
:1038400001E0D3D0012BEFD7016B0151106E116A4B
:10385000D890115004E6CE0E105C000E115802E212
:10386000ABD9F3D7036B5FD90B010051330A62E088
:10387000CC0A5DE0C90A47E0350A23E0020A0DE000
:10388000340A01E07DD04FD90B01000501E0ADD035
:103890000101020E376F0B0E48D072D901E0A5D09E
:1038A0000101100E376F030E49D9110E376F030E49
:1038B00045D9120E376F030E41D9130E376F030E21
:1038C00034D05ED901E291D001010C0E376F030EA6
:1038D00035D90D0E376F030E31D90E0E376F030E2B
:1038E0002DD90F0E376F030E50D9040E0B01005F58
:1038F0000B0100510007000952E00101010E376F72
:103900000B0E43D9F5D73CD970E10101070E376F93
:103910000B0E14D9060E376F0B0E10D9050E376F2C
:103920000B0E0CD9040E376F0B0E2FD938D0010EA9
:10393000036F35D025D959E10101070E376F030E0A
:10394000FDD8060E376F030EF9D8050E376F030E3C
:10395000F5D8040E376F030E18D9D880080E03016E
:103960000455070E0555000E0655000E075517E2C3
:10397000080E045F070E055B000E065B075B0FD0A9
:103980000101000E376F0B0E00D90B01005100072B
:10399000000905E00101010E376F0B0EF5D70B0191
:1039A000035101E160D7020E025D09E104CB00F38F
:1039B00005CB01F306CB02F307CB03F311D0000EC6
:1039C000E96E030EEA6EEE50041908E1EE50051997
:1039D00005E1EE50061902E1EE50071901E0026B15
:1039E00035EC19F00B010251120035EC19F0000C06
:1039F0000101010E9ED8010E9CD8060E9AD8ABD8B4
:103A0000120E97D8230E95D8340E93D8560ECBD8D5
:103A1000800EC9D8A0D89FD8316B14EC18F00B01D8
:103A2000196B0C0E195D02E2A0D8FBD7BCC231F1B4
:103A300014EC18F0BDC231F114EC18F0BEC231F133
:103A400014EC18F0BFC231F114EC18F0C0C231F11F
:103A500014EC18F0C1C231F114EC18F00B01196B21
:103A60001951106E116AD890115004E6CA0E105CFC
:103A7000000E115802E279D8F3D70101630E59D82C
:103A8000820E57D8530E55D8630E53D8350E51D8E1
:103A9000010E316F14EC18F016C331F114EC18F06C
:103AA0000301160518E0085109110A110B1113E062
:103AB0000101360E7CD803C331F114EC18F002C3B7
:103AC00031F114EC18F001C331F114EC18F000C31B
:103AD00031F114EC18F00101370E2BD8020E29D861
:103AE000010E27D8030E316F14EC18F0030E0301FA
:103AF000165D13E10101320E5AD808C331F114ECFE
:103B000018F009C331F114EC18F00AC331F114ECC8
:103B100018F00BC331F114EC18F00101316914EC09
:103B200018F079EF18F00101000E376F0B0EC5EF9A
:103B30001DF0316F14EC18F00101120026D80101BC
:103B40001200030114510301645D106E65510301FD
:103B50001555116E1200316B14EC18F001011200B2
:103B600064C314F365C315F312000101316B14EC47
:103B700018F00B01192B120076C32FF107EF18F084
:103B8000D2DF040E0B01005D1200386FE7EF18F072
:103B9000166F2EDFE5DF03011200D3DF900E105CFD
:103BA000FF0E11581200C5DFD6DFABEF1DF0C1DFED
:103BB000040E316F14EF18F0B6DF0B01012B120069
:103BC0000001F35101E112000001FB0EF16F5C0EE8
:103BD000F26FEAEC32F000010B0EF16F5B0EF26F48
:103BE000EAEC32F0F3C0B4FB0B01B451000814E26C
:103BF000B451070B05E100012E0EED6F8BEC32F096
:103C000027DA02E057D908D0320EE66E85EC34F0A0
:103C1000E5520B01B407E8D72DEF20F03CDAE7D9E5
:103C2000010EE926000EEA22E2D9020EE926000E74
:103C3000EA22DDD9030EE926000EEA223EEF20F04B
:103C40000B01016B05DAFEE07BEC32F00B01006F3B
:103C50000D0E005D17E00A0E005D14E0012B00015F
:103C6000F6C0E9FFF7C0EAFFF62B000EF72300CB02
:103C7000EFFFF6C0E9FFF7C0EAFFEF6AF851F80777
:103C80000009E0E10B0101511200F9C001FBFAC08B
:103C900002FB0B01036BF9C0E9FFFAC0EAFFEFCFAB
:103CA00000FBEF5021E02E0E0B01005D11E1000141
:103CB000F9C0E9FFFAC0EAFFF92B000EFA23EF6A18
:103CC000AFD9032BD1D9F9C001FBFAC002FB07D051
:103CD000300E005D03E30051390801E2000C0001E1
:103CE000F92B000EFA23D7D79BD9BED9030E0B01AF
:103CF000035D01E0000C010CABD9FEE07BEC32F07F
:103D00000B01006F310E005D05E3390E005D02E22C
:103D100000511200390CA1D9300E0001FD5DFF0FDA
:103D2000E96EEA6AD890E936EA362D0EE926030EE6
:103D3000EA22EECFF1F0EDCFF2F0EAEC32F0000142
:103D4000FD51380A01E1B5D00F0A01E1B0D0010AF6
:103D500001E1A1D0030A01E197D0010A54E0070A6A
:103D60004BE0010A42E0030A01E012000201330EB7
:103D7000D66F94EC31F00B01A16F0201340ED66FB7
:103D800094EC31F00B01A26F870EE66E0B0EE66E1F
:103D9000A1CBE6FFA2CBE6FF87D9870EEF6F0B0E14
:103DA000F06FD9EC32F029D9000947E0870EE66EB2
:103DB0000B0EE66E5EEC2BF0E552E552F3CFA1FB65
:103DC000F4CFA2FBF3CFA8FF0201330ED76F9EEC16
:103DD00031F0A2CBA8FF0201340ED76F9EEC31F078
:103DE000A2CBC0F2A1CBC1F212000B01B80E9F6FA3
:103DF000020EA06FA36B0ED00B01C60E9F6F020EBA
:103E0000A06F0E0E06D00B01C20E9F6F020EA06FA8
:103E10000A0EA36F9FCBF4F0A0CBF5F0FFDEEDD838
:103E200000019B0EFB6F0B0EFC6F0001870EF96FFC
:103E30000B0EFA6F2ADF00090BE10001B10EF16FE2
:103E40005C0EF26FEAEC32F003D9FEE07BEF32F069
:103E50009FCBE9FFA0CBEAFF9BCBEEFF9CCBEEFF15
:103E60009DCBEEFF9ECBEEFF9BCBA8FFEAD89CCB71
:103E7000A8FFE7D89DCBA8FFE4D89ECBA8FF0B01F5
:103E8000A351A32B020110D00201160ED66F94ECA1
:103E900031F0010906D00201160ED66F94EC31F014
:103EA000FE0BA86E0201160ED76F9EEF31F06FEF7A
:103EB0001FF012000001440EF16F5B0EF26FEAEC8E
:103EC00032F01ADF0B01B56F390EB55D03E0B5CBEB
:103ED000FDF021DF380E0B01B55DECE112000B01A6
:103EE000006B026BF8EC23F064C385FB65C386FBB3
:103EF0000B0185510301645D106E65510B01865500
:103F0000116E320E105C000E115809E364C385FB7C
:103F100065C386FB0001150EED6F8BEC32F098D86F
:103F2000E7E00B01025162E193D8FBE07BEC32F059
:103F30000B01016F0051030A20E0010A1BE0030A94
:103F400014E0010502E1010E16D0040E015D09E145
:103F500041EC24F00001060E9BD80B01010E026F0C
:103F6000E0D70001150E94D8DCD7060E046F036B62
:103F7000020E01D0030E006FD4D70351032BEA6A5F
:103F8000050FE96E0B0EEA2201CBEFFF0351106E15
:103F9000116A1134C6E210508008000E1154C1E2BB
:103FA000060E046F016B0151106E116AD89011500A
:103FB00004E6800E105C000E11580DE20151EA6A11
:103FC000050FE96E0B0EEA22EFCF45F210EC24F05C
:103FD0000B01012BE8D70201376B68EC23F004CB0F
:103FE000EDF08BEC32F00B01006B9BD7010C46D847
:103FF00000012E0E4DD84BEF20F00001290E48D8BD
:1040000000013A0E45D80001200E42D80001140EDE
:10401000F86F0001870EF66F0B0EF76F20EF1EF0A2
:1040200001CBE6FF02CBE6FF5EEC2BF0E552E5525A
:10403000F350E66EFBC010F0FCC011F00B01035111
:1040400012000B01A351A32B0201D76F9EEF31F099
:104050000001EA510001EB5D120000010D0E18D8BD
:1040600000010A0E48EF20F00F011024E96E000E47
:104070001120EA6EE552E750EF6E1200EF50E66E47
:10408000E66A12D8000EEF6F0B0EF06FD9EF32F028
:10409000ED6F8BEF32F0000EE66E0B0EE66EF4C0A5
:1040A000E9FFF5C0EAFF1200D3EC2BF0E552E55230
:0840B000E552E5520001120087
:0840B800150E01014F6F506B62
:1040C0006EEC00F00101936F976BC56B926B140E51
:1040D000956F966B120093C155F12CEC01F000091D
:1040E00007E10101C56B070E996F976B926BA6D024
:1040F00093C169F144EC03F0000934E020DA0101D6
:10410000700E626F0B0E636F93C161F1B9EC02F038
:1041100000090EE01F0E0101C55DF1E2C551C52B7E
:10412000EA6AA40FE96E010EEA2270CBEFFFE7D72F
:1041300093C160F19BEC02F00A0E0B01705D26E169
:104140000101C551EA6AA40FE96E010EEA22EF6A85
:10415000C56B9BD9C6C1D8F1C7C1D9F15DD90101E1
:10416000996F14D00101975111E0D5510301645D9D
:10417000106E65510101D655116E500E105C460E41
:10418000115804E3DCD9020E996F976F0101975122
:10419000020A3EE0070A0DE0040A06E0010A54E1C3
:1041A0009A6BCDD9010E976FBED94EE00101050E75
:1041B000976FB9D92DE09AC1E9FFEA6AE9BEEA68CA
:1041C000D890E936EA36A20EE926020EEA22EECFB0
:1041D00071FBEDCF72FB0B0171CBF6FF72CBF7FFDA
:1041E000712B000E72230800F5CF70FBF55007E02D
:1041F00070CB5AF193C159F1F2EC01F0ECD793C1B5
:1042000057F175EC01F001010B0E9A6F020E976FDA
:10421000070E0101995D18E099C1D7F116D8000980
:104220000FE00B0E01019A5D02E0050E04D0020EB4
:10423000995D02E1010E976F070E996F986B010C63
:104240000B0E01019A5DB3E1010C0101D751050A82
:1042500051E0060A4DE0070A34E0060A30E0030A9E
:1042600018E0010A51E192819293010E9A6F090EB2
:10427000E66EE66AC8C1E6FFC9C1E6FF9B0EE66EC0
:10428000010EE66E33EC31F0106E060EE15E10505A
:10429000010C92A112D0C8C16FF3C9C170F3030120
:1042A0009B0E6D6F010E6E6F5EEC2FF0000904E047
:1042B00001019283020E29D00101060E26D087EF5C
:1042C00021F0D0C1E6FFD1C1E6FF5EEC2BF0E55254
:1042D000E552F3CF96F1D2C1E6FFD3C1E6FF5EEC23
:1042E0002BF0E552E552F3CF95F101010A0E0DD006
:1042F000B0EF21F00A0E9A6FFE0E945D07E094C1B4
:1043000056F135EC01F0010C050E9A6F010C01011C
:104310009851030A18E0020A0FE0010A20E1020E98
:10432000985D02E141EC24F0FE0E0101945D06E08F
:1043300010D90101010E05D0FCD811E10101030ED5
:104340009A6F986F000CEFD80AE093C155F12CECEE
:1043500001F0000904E093C156F135EC01F0000CC6
:1043600001019851020A2EE0030A21E0010A53E1FB
:1043700092B302D0060E4DD0070E9A6F95C153F13D
:1043800096C154F19351220DF3CFE9FFF4CFEAFF28
:10439000000EE9260C0EEA22EE52E9CF51F1EACFE7
:1043A00052F1AAEC00F00101946F010E09D0C1D8BE
:1043B00032E0020131A12FD0F8EC23F00101020E0E
:1043C000986F000C94C169F144EC03F000091AE005
:1043D000B6D80101730E626F0B0E636F94C161F169
:1043E000B9EC02F0000905E073CB45F210EC24F0C3
:1043F000F0D70201376B68EC23F094C160F19BECBD
:1044000002F0000C96D807E1A4D80101FE0E946FCB
:10441000090E9A6F010C000C0B01006B060EE76E83
:104420000019E8AE02D0E73402D0E750005D2CE27C
:10443000040EE66EE66A00CBE9FFEA6AE9BEEA68C6
:10444000D890E936EA36960EE926020EEA22EECF39
:1044500010F0EFCF11F0126A10C0E6FF11C0E6FFB6
:1044600012C0E6FFD8C1E6FFD9C1E6FF89EC30F003
:10447000136E070EE15E1350000903E10B010051BA
:1044800012000B01002BCAD7060C0B01036BA40E04
:10449000006F010E016F58D8EF50200804E1002B87
:1044A000000E0123F8D700CBC6F101CBC7F1010103
:1044B000010ED46F49D8EFCF02FBEF5033E00B0170
:1044C0000351010A16E0010A29E1200E025D03E012
:1044D0002C0E025D05E138D8EF6A010E036F1ED085
:1044E0000D0E025D03E00A0E025D18E12DD8EF6AA1
:1044F00015D0200E025D12E00101D451D42BE96EDB
:10450000EA6AD890E936EA36C60EE926010EEA22B2
:1045100000CBEEFF01CBEDFF0B01036B002B000E78
:104520000123C8D7120093C158F1D9EC01F000095A
:10453000120094C155F12CEC01F00009120064C383
:10454000D5F165C3D6F1120000CBE9FF01CBEAFF3C
:0E455000120041EC24F094C156F135EF01F059
:02455E00020158
:10456000306B010E316F0301180E3D6F89EC2FF097
:104570000B01006B060E005D05E2005191D9EF6A58
:10458000002BF8D7010C0B01FE0E026F020131A1C6
:10459000FE0C0B01016B060E015D0AE2015180D990
:1045A000EF50010B03E101CB02FB02D0012BF3D74B
:1045B000FE0E025D01E1FE0C450E036F046B056B00
:1045C00033C2E9FF34C2EAFFEF5001E1FF0C33C20E
:1045D000E6FF34C2E6FF61EC31F0E552E552F3CF7D
:1045E00033F2F4CF34F203CB42F304CB43F367D975
:1045F00004E00B01FE0E026F5ED013EC30F00B01F5
:10460000006F00AF02D0026956D0016B0C0E015D45
:1046100021E213EC30F00B01006F01510201EA6A54
:104620003325E96E3451EA22EF500B01005D06E0BC
:10463000120E0327000E042305230CD0005108E1BD
:104640000B01012B0C0E015D05E213EC30F0F8D7E5
:10465000012BDCD70C0E015D2BE10251080DF3CFCD
:1046600006FBF4CF07FB000E0627020E072333D903
:10467000010EEF6E30D9EB6A020EEB6A13EC30F0EC
:10468000E66E29D9030E03D9030E2AD9010EFFD8ED
:10469000030E26D9020EFBD8060EF9D8060E20D935
:1046A000010E1ED9E552E750EF6E0201302B03D008
:1046B0001DEC30F098D71DEC30F00B0102511200C8
:1046C00036C237F205D802013651EAD8EF6A120035
:1046D00002013751080DF3CFAFFBF4CFB0FB000E52
:1046E0000B01AF27020EB023F1D8EF50020B03E00D
:1046F0001DEC30F00DD0EAD8EF50040B09E009ECC6
:1047000030F00301A00E4B6F58EC30F00009F9E1D6
:10471000F90EDCD8E850EF160201319312000201C5
:104720003851080DF3CF01FBF4CF02FB000E0B0153
:104730000127020E02239F0E106EBCD8E850EF1620
:10474000B9D8EF50010B25E0B5D8EF50020B24E1AA
:10475000020131B31ED0AED8EE52EECF13F0EFCF40
:1047600014F0156AA7D8030EBBD8EE501324106EB0
:10477000EE501420116EEE501520126E10C042F350
:1047800011C043F39CD805E195D8EF820201318333
:1047900003D090D8EF8A000C13EC30F00B01006FBF
:1047A00089D8EE52EE2A000EED22EECF10F0EDCFBA
:1047B00011F080D8060E94D8EECF12F0EFCF13F0A0
:1047C00000011250101805E11350111802E172D8BF
:1047D000EF8C0B0100511200010C010C12001200B1
:1047E000F36AF46A1200056A066A076A1200000C8E
:1047F000020131A1000C0B01AF6B060EAF5D08E2A8
:10480000AF514ED8EF50010B01E0000CAF2BF5D7A4
:104810000201010E006F400E036F046B056B010C6B
:104820000B01000EB16F020EB26F020100A506D09F
:10483000400E325D03E30201376B4ADF020100B52F
:1048400015D031A302D0008B000C03C23FF304C289
:1048500040F30301A00E3E6F92EC2FF0000905E13A
:10486000020100853183326B01D0000C45C244F354
:10487000F5EC2FF00201322B032B000E042305234D
:10488000010C0201376B24DF0201006B010C28D8F8
:10489000E552E750EF6E13EC30F0E66E6BEF24F06C
:1048A000080DF3CFE9FFF4CFEAFF000EE926020E70
:1048B000EA22120001CBE9FF02CBEAFF120003015A
:1048C000A00E416FC8EC2FF000091200AFCBE9FF3A
:1048D000B0CBEAFF120006CBE9FF07CBEAFF1200DC
:0848E000E926000EEA22120095
:0848E800D9C2F3FFD8C2F4FFAE
:1048F0001200DAC201FBDBC202FBDCC203FBDDC239
:1049000004FB0B01010E056F0B0E066F05CBE9FFD3
:10491000EA6E030E9AD9EF50E66E030E90D900CBE3
:10492000EFFF84D9020E91D9010E85D9EF50E66EC2
:104930007DD9020E84D9010E7ED900CBEFFF01CBC9
:1049400004F002CB05F003CB06F004CB07F0120015
:104950000B01406B416B426B436BDEC23EFBDFC21F
:104960003FFBE0C23CFBE1C23DFBD8903D333C3312
:104970003CCB10F03DCB11F03C07000E3D5B1050DE
:10498000111018E03ECBE9FF3FCBEAFF020E3E27B5
:10499000000E3F23EECF10F0EFCF11F000011050CA
:1049A0000B014027000111500B014123000E42234F
:1049B0004323DED70201E051010B0EE03ECBE9FFBD
:1049C0003FCBEAFFEFCF10F0000110500B01402762
:1049D000000E4123422343230B014251431109E0BE
:1049E00040514225406F41514321416F426B436B1F
:1049F000F3D740CB10F041CB11F0101E111E10C0A8
:104A0000F3FF11C0F4FF12000B01010E006F016BE8
:104A1000026B0201E251E3114EE0400EE25D000E36
:104A2000E35904E3400E106E116A04D0E2C210F0A4
:104A3000E3C211F010C005FB0B0110500201576FCB
:104A4000586B0201060E556F0B0E566F20EC15F0D9
:104A50000B010551106E116A10500201E25F1150F6
:104A6000E35B0B01046B0551045DD3E20451EA6A78
:104A7000060FE96E0B0EEA22EFCF03FB00510AE1AD
:104A800003510125016F0351015D0DE2022B0BE182
:104A9000012B09D003510225026F0351025D03E28D
:104AA000012B01E1022B005102E0000E01D0010EAA
:104AB000006F042BD8D70B01021D026F011DF36E8E
:104AC00002CBF4FF12000201E451390805E3300E75
:104AD000E45D02E3300E0FD0E451460805E3410ED9
:104AE000E45D02E3370E07D0E451660806E3610E89
:104AF000E45D03E3570EE45D1200FF0C010E0201BA
:104B0000EA6AE525E96EE651EA22EFCFE4F2DBDF5F
:104B10000B01236FE5C2E9FFE6C2EAFFEFCFE4F243
:104B2000D2DF0B01246FFF0E235D03E0FF0E245D37
:104B300001E1000C2439F00B2311E7C2E9FFE8C2C0
:104B4000EAFFEF6E010C0B01236BA6B2FED72F0E0E
:104B5000A616A6840201EBC2E9FFECC2EAFFEB2B2A
:104B6000000EEC23EF50A86E0B01232B0201ED5138
:104B70000B01D880235501E2A86AEAC210F0116A3D
:104B80001050AA6E0201E9C210F0EAC211F0E92B3E
:104B9000000EEA231050A96E550EA76EAA0EA76E3E
:104BA000A6820000A6B2FED7A850D4E1A6940B01BD
:104BB000235100D01200F1C210F01050AA6EF0C2C2
:104BC000A9FF3F0EA6160201EEC2E9FFEFC2EAFFFF
:104BD000EE2B000EEF23EFCF1CFBA680A8500B019D
:104BE0001C5D01E0010C1C5101E1000CA92AEBE164
:104BF000AA2AE9D7F2C202FBF3C203FB0B01006B46
:104C0000016B0201F4510B01005D0201F5510B0132
:104C100001590BE202CBE9FF03CBEAFF022B000EA6
:104C20000323EF6A002B0123ECD7120005CBE9FF29
:104C300006CBEAFF1200E926000EEA221200FBDF93
:104C4000E552E750EF6E16EF26F0F5DFEFCF00FBF1
:044C500016EF26F045
:0C4C5400140E0201576F586B0201080E8D
:104C6000556F0B0E566F20EC15F0F00E0B0108156A
:104C7000400801E0A1D00F0E0815040DF350106E8E
:104C8000116A140E105E000E115A10C01CFB105059
:104C9000140801E291D01C5100080BE21C510201E2
:104CA000576F586B02011D0E556F0B0E566F20EC9F
:104CB00015F012CB00FB13CB01FB0B01126B136B36
:104CC000140E16D9080EDE6F0B0EDF6FA8EC24F061
:104CD000F3CF04FBF4CF05FB0B01041F051F1C5190
:104CE000000810E21C5104D91D0EDE6F0B0EDF6FA1
:104CF000A8EC24F0F3CF06FBF4CF07FB0B01061F53
:104D0000071F02D0066B076B040EF2D8040EDE6F8D
:104D10000B0EDF6FA8EC24F0F3CF02FBF4CF03FB04
:104D20000301080E596F0B0E5A6FB5D80B010251D3
:104D3000001942E1035101193FE1F00E0815400846
:104D40003BE103014C514D110CE04CC3E9FF4DC355
:104D5000EAFF18CBEEFF19CBEEFF1ACBEEFF1BCB11
:104D6000EEFF4EC3E9FF4FC3EAFF060EDBD814CBBC
:104D7000EEFF15CBEEFF16CBEEFF17CBEEFF50C3C9
:104D8000E9FF51C3EAFF11CBEFFF0B011C51126E7B
:104D9000136A12500A5D106E13500B59116E140EE7
:104DA000105E000E115A52C3E9FF53C3EAFF10C050
:104DB000EEFF11C0EDFF010C7AEC15F0000C0B01B9
:104DC000450E286F296B140E030157250B012A6F1E
:104DD000000E030158210B012B6F0101FD2B000E6A
:104DE000FE23FDC12CFBFEC12DFB0B012E6B400EE3
:104DF0002F6F640E306F56C331FB326B336BB8C20A
:104E000034FBB9C235FBBAC236FBBBC237FB54C355
:104E1000E9FF55C3EAFF060E85D8EECF38FBEECF8B
:104E200039FBEECF3AFBEFCF3BFB0301280E596F66
:104E30000B0E5A6F30D8140E5BD8280EDE6F0B0E97
:104E4000DF6FA8EC24F0F3CF32FBF4CF33FB140E6A
:104E5000030157250201626F000E03015821020170
:104E6000636F0201616B54C3E9FF55C3EAFF54C38A
:104E70005FF255C360F272EC16F0140E0201536F2C
:104E8000546B0201280E516F0B0E526F64EC14F03C
:104E9000F36AF46A120027D8020E35D8020E38D809
:104EA000020E2BD8020E39D8040E2DD8040E30D89D
:104EB000040E23D8040E31D8060E25D8060E28D8A5
:104EC000060E1BD8060E29D80A0E1DD80A0E20D8A9
:104ED0000A0E13D80A0E03D83CCBEFFF120022D8DB
:104EE000010E92EF27F059C3E9FF5AC3EAFF1200FF
:104EF0000201E06FE16B0201120014D8E552E750A5
:104F0000EF6E73EF27F00ED8EFCF3CFB73EF27F077
:104F1000E6DFEF50E66E73EF27F0E1DF3CCBEFFF0B
:0C4F200073EF27F0E926000EEA221200D1
:044F2C004854545041
:104F30002F312E3020353033200D0A0D0A53657283
:104F40007669636520556E617661696C61626C6536
:104F50000D0A000D0A0D0A00485454502F312E300E
:104F600020323030204F4B0D0A436F6E74656E74E3
:104F70002D747970653A2000485454502F312E30EA
:104F800020343034204E6F7420666F756E640D0AC5
:104F90000D0A4E6F7420666F756E642E0D0A0061E7
:104FA0007564696F2F782D77617665006170706C1C
:104FB00069636174696F6E2F6A6176612D617263D6
:104FC0006869766500696D6167652F6A706567005D
:104FD000696D6167652F67696600746578742F6A0B
:104FE00061766173637269707400746578742F639D
:104FF0007373006170706C69636174696F6E2F6A9E
:105000006176612D766D00746578742F68746D6CAF
:1050100000746578742F706C61696E0047756573F4
:1050200074004E6F00537570657220557365720081
:105030000D0A4E6F772072756E6E696E6720617013
:10504000706C69636174696F6E2E2E2E000D0A52AA
:105050006561647920746F20646F776E6C6F616432
:105060002046696C652053797374656D20496D61C4
:105070006765202D2055736520586D6F64656D2020
:1050800070726F746F636F6C2E0D0A000D0A4448C6
:105090004350202620495020476C65616E696E6739
:1050A0002064697361626C65642E0D0A000D0A4408
:1050B000484350202620495020476C65616E696E38
:1050C0006720656E61626C65642E0D0A000D0A44EE
:1050D000656661756C74205375626E6574204D61F0
:1050E000736B2028000D0A44656661756C74204757
:1050F00061746577617920416464726573732028F7
:10510000000D0A44656661756C7420495020416445
:1051100064726573732028000D0A53657269616CAF
:10512000204E756D626572202800323030206F6B22
:105130000D0A00323236205472616E736665722039
:10514000436F6D706C6574650D0A00313235204413
:105150006F6E652E0D0A00313530205472616E730A
:1051600066657272696E6720646174612E2E2E0D01
:105170000A00353330204C6F67696E207265717597
:10518000697265640D0A00353032204E6F742069F3
:105190006D706C656D656E7465640D0A0035303038
:1051A000200D0A00323231204279650D0A00323377
:1051B00030204C6F6767656420696E0D0A003333D9
:1051C000312050617373776F7264207265717569F5
:1051D0007265640D0A003232302052656164790DC7
:1051E0000A0041424F5200504F52540053544F5204
:1051F00000515549540050415353005553455200F6
:105200001C0E0201576F586B0201000E556F0B0EFA
:10521000566F20EC15F07AEC15F00301000E626F6A
:105220000B0E636FF5D80B01010E001912E101514D
:1052300010E10451106E116A060E10180AE11150A7
:1052400008E10551126E136A040E121801E11350A1
:1052500001E0000C020E061905E1075103E106D931
:10526000EF6A0DD0010E061906E1075104E1010EA7
:10527000FDD8EF6E04D0020EF9D8EF6E000C0201DB
:10528000B8510B01185D2EE10201B9510B01195DF6
:1052900029E10201BA510B011A5D24E10201BB515F
:1052A0000B011B5D1FE15BC3E9FF5CC3EAFF08CB99
:1052B000EEFF09CBEEFF0ACBEEFF0BCBEEFF0CCBE4
:1052C000EEFF0DCBEEFF5BC3E9FF5CC3EAFF060E0A
:1052D000D7D80ECBEEFF0FCBEEFF10CBEEFF11CBEE
:1052E000EEFF010C000C010E0B01006F016B026B55
:1052F000080E036F060E046F040E056F03016105AF
:105300000BE1010E0B01066F076B1269136914693B
:1053100015691669176914D0020E0B01066F076B29
:105320005FC3E9FF60C3EAFFEECF12FBEECF13FBD2
:10533000EECF14FBEECF15FBEECF16FBEFCF17FB36
:10534000BCC208FBBDC209FBBEC20AFBBFC20BFB4D
:10535000C0C20CFBC1C20DFBB8C20EFBB9C20FFB31
:10536000BAC210FBBBC211FB7AD8EF500E19020172
:10537000C2151BE174D8010E83D8EF500B010F1931
:105380000201C31512E16BD8020E7AD8EF500B015F
:1053900010190201C41509E162D8030E71D8EF504B
:1053A0000B0111190201C51509E0C6C218FBC7C2DD
:1053B00019FBC8C21AFBC9C21BFB09D050D8EECFDB
:1053C00018FBEECF19FBEECF1AFBEFCF1BFB03014F
:1053D000000E626F0B0E636F1BD81C0E0201626F12
:1053E000636B0201060E616F0201120E5F6F0B0EFE
:1053F000606F72EC16F01C0E0201536F546B0201C9
:10540000000E516F0B0E526F64EC14F0C9EF16F0E2
:1054100032D819D8F3CFEEFF11C0EDFF2CD8020E11
:105420002FD811D8020EF3CFEBFF030E11C0EBFF04
:1054300022D8060E25D807D8060EF3CFEBFF070EAD
:1054400011C0EBFF1200EECFD8F2EDCFD9F274EC21
:1054500024F0F3CF10F0F4CF11F03BEF2AF05FC34C
:10546000E9FF60C3EAFF060E40EF2AF05DC3E9FFE3
:105470005EC3EAFF120062C3E9FF63C3EAFF1200E2
:08548000E926000EEA221200E9
:085488000D01BD6BBE8171EC4A
:1054900013F0FCEC32F0ADEC17F03AEF00F00B013A
:1054A000010EB46F0B01B45101E1FDD0B46B0D01DD
:1054B000BD51040A01E1D7D0070A01E1A1D0050AD4
:1054C00001E187D0010A72E0050A3FE0070A36E0F1
:1054D000050A02E0010AE6E10201B30E5D6F0B0E60
:1054E0005E6F0201BF0E5B6F0D0E5C6FBFEC15F0BF
:1054F000000915E10201160ED66F94EC31F0010B94
:10550000D1E0B1EC15F00009CDE10201B86BB96B47
:10551000BA6BBB6B0D01BE810CEC1BF0C3D70B014A
:10552000010EB46FB35103E10D01020E39D0060E26
:10553000B35D01E095D00D01050E32D00B01B46BC7
:1055400009EC33F00009AEE0ABD00301C90E526F95
:105550000D0E536F0301B30E506F0B0E516F03010D
:10556000BF0E4E6F0D0E4F6F0301AF0E4C6F0B0E43
:105570004D6F2AEC26F0000916E00B01010EB46F06
:10558000B30503E10D01030E0BD0060EB35D03E17D
:105590000D01060E05D0110EB35D04E10D01070EDD
:1055A000BD6F80D7B46B7AEC15F07AD0C9CD41F1DC
:1055B000CACD42F10101AF0E3F6F0B0E406F0101EA
:1055C000BF0E3D6F0D0E3E6F3DEC19F0000915E06A
:1055D00012D0C9CD6EF1CACD6FF10101AF0E6C6F63
:1055E0000B0E6D6F0101BF0E6A6F0D0E6B6F2DEC10
:1055F00004F0000902E00D01BD6B0B01B46B52D742
:10560000BD6B290ED880C955000ECA5529E3030188
:10561000ED0E1F6F0D0E206F0301EB0E1D6F0D0EB3
:105620001E6F0301C90E1B6F0D0E1C6F0301CB0E05
:10563000196F0D0E1A6F0301B30E176F0B0E186F53
:105640006DEC2CF000090AE0080E0B01B35D06E1D9
:10565000010EB46F0D01040EBD6F02D00D01BD6BC4
:105660007AEC15F01FD734EC14F0000901E11AD7D9
:10567000EDCD29F3EECD2AF3EBCD27F3ECCD28F3D6
:10568000C9CD26F30301CB0E246F0D0E256F030148
:10569000236B0301BF0E216F0D0E226FE7EC2CF080
:1056A0000D01BD6BFFD651EC03F01AEC1BF00301AA
:0C56B00077A102D00D01BE911EEF14F096
:0456BC00FF0EE3CF2B
:1056C000EAFFE552FF0EE3CFE9FFE552E66AE66A3C
:1056D000D9CFE6FFDACFE6FFFC0EE124D96EFF0E4C
:1056E000E220DA6EE66AE66AE66A200EEF5C06E021
:1056F000090EEF5C03E0EF6603D03FD0EE50F5D724
:105700002D0EEF5C03E1FF0EE32A03D02B0EEF5CBE
:1057100001E1EE502F0EEF6424D03A0EEF6021D05D
:10572000D890F90EE336FA0EE336FD0EDECFE3FF36
:10573000FE0EDDCFE3FFD890F90EE336FA0EE33626
:10574000D890F90EE336FA0EE336FD0EE350DE266E
:10575000FE0EE350DD22300EEE5CDE26000EDD2272
:10576000D9D7FF0EE3CFE8FFE85207E0F90EE31EBA
:10577000E32AFA0ED8B4E306E31EE552E552E552F9
:10578000FF0EE3CFDAFFE552FF0EE3CFD9FFE5527C
:10579000E1CFE9FFE2CFEAFFED52ED52EECFF3FFAA
:1057A000EFCFF4FF1200D9CFE6FFDACFE6FFFA0E13
:1057B000E3CFD9FFFB0EE3CFDAFFFD0EE35209E79B
:1057C0002D0EDE6EFC0EE31EE32AFD0ED8B4E306BA
:1057D000E31EE652E652E652FD0EE124E76EFF0EAE
:1057E000E220E46EE652F70EE3CFE6FFF70EE3CFDA
:1057F000E6FF43EC2CF0F90EE124E96EFF0EE22007
:10580000EA6E33EC2CF00AE130EC2CF009E133ECD9
:105810002CF008E130EC2CF007E108D03EEC2CF045
:1058200039EC2CF03EEC2CF039EC2CF03EEC2CF06A
:10583000DE6AF90EE126FF0EE222FF0EE3CFDAFF69
:10584000E552FF0EE3CFD9FFE552FC0EE124E96EED
:10585000FF0EE220EA6EEECFF3FFEFCFF4FF12006F
:10586000EF380F0B1200EF500F0B02E1EE52D8840D
:105870001200EF380F0B300FDE6E1200EE500F0BE0
:10588000300FDE6E1200FC0EE3CFE9FFFD0EE3CF1A
:10589000EAFF100EE66EEE6AEE6AEF6AD890FD0E31
:1058A000E336FE0EE336ED36ED36EF36FF0EE30659
:1058B00009E064EC2CF0EE5264EC2CF0EE5264EC57
:1058C0002CF0EDD7E56E1200030EEF24E8B6EF6E74
:0A58D000300EEF24E8BEEF6E000C6E
:0658DA00080E0201576FE9
:1058E000586B0201000E556F0B0E566F20EC15F031
:1058F00002CB2EFB03CB2FFB0B01026B036B080EBD
:105900000201E06FE16B0201000EDE6F0B0EDF6F34
:10591000A8EC24F0F3CF28FBF4CF29FB0B01281FC0
:10592000291F080E106ED9D8E850EF5ED6D8EF5078
:105930000201576F586B19C355F21AC356F220EC87
:1059400015F0CBD8EF500201E06FE16B19C3DEF226
:105950001AC3DFF2A8EC24F0F3CF2AFBF4CF2BFB21
:105960000B012A1F2B1F040E0201E06FE16B0201E5
:10597000280EDE6F0B0EDF6FA8EC24F0F3CF2CFBAC
:10598000F4CF2DFB0301000E2B6F0B0E2C6F7AD87A
:1059900017C3E9FF18C3EAFF00CBEFFF1DC3E9FF00
:1059A0001EC3EAFF04CBEEFF05CBEDFF1FC3E9FFEB
:1059B00020C3EAFF06CBEEFF07CBEDFF0B012E5114
:1059C0002C1902E12F512D1901E0000C010C0B01E3
:1059D000016B23C300FB026B036B27C304FB28C3CB
:1059E00005FB29C306FB2AC307FB03012651E66E0C
:1059F000E66A24C3E6FF25C3E6FF080EE66E0B0E3B
:105A0000E66EA8EC30F0106E060EE15E1050030159
:105A1000000E2B6F0B0E2C6F35D8080E03012625B8
:105A20000201E06FE16B000EE1230201000EDE6F68
:105A30000B0EDF6FA8EC24F0F3CF02FBF4CF03FBD7
:105A4000080E030126250301576F586B000E5823DB
:105A50000301010E566F21C354F322C355F3DFEC4B
:105A600026F0080E030126250201536F546B000E29
:105A700054230201000E516F0B0E526F64EC14F0B0
:105A8000C9EF16F02FD8040E15D8040EF3CFEBFF94
:105A9000050E1FD8060E0ED8060EF3CFEBFF070E2D
:105AA00018D8020E07D8020EF3CFEBFF030E11C079
:105AB000EBFF1200E926000EEA22EECFD8F2EDCF7E
:105AC000D9F274EC24F0F3CF10F0F4CF11F072EFB0
:105AD0002DF011C0EBFF72EF2DF01BC3E9FF1CC3CB
:0E5AE000EAFF12002BC3E9FF2CC3EAFF1200FD
:025AEE004D6FFA
:105AF0006474726F6E6978205443502F495020535C
:105B00007461636B2056332E3033000D0A5072657A
:105B1000737320616E79206B657920666F72204304
:105B20006F6E66696775726174696F6E206D656E00
:105B3000752E00444843502F476C65616E696E674F
:105B40002E2E2E000D0A0D0A0D4D785765625372E8
:105B500076722044656D6F204170706C696361746A
:105B6000696F6E2076312E3020284D6F6474726F0D
:105B70006E6978205443502F495020537461636BF1
:105B80002056332E30332C204665622032322032AC
:105B9000303036290D0A0D0A09313A204368616E0A
:105BA000676520426F6172642073657269616C2061
:105BB0006E756D6265722E0D0A09323A2043686176
:105BC0006E67652064656661756C7420495020615C
:105BD0006464726573732E0D0A09333A2043686159
:105BE0006E67652064656661756C742067617465B5
:105BF00077617920616464726573732E0D0A0934CC
:105C00003A204368616E67652064656661756C74EF
:105C1000207375626E6574206D61736B2E0D0A09B9
:105C2000353A20456E61626C652044484350202619
:105C300020495020476C65616E696E672E0D0A0918
:105C4000363A2044697361626C65204448435020B1
:105C50002620495020476C65616E696E672E0D0ADB
:105C600009373A20446F776E6C6F61642046696C27
:105C7000652053797374656D20496D6167652E0DDC
:105C80000A09383A205361766520262051756974D7
:105C90002E0D0A0D0A456E7465722061206D656EC9
:105CA000752063686F6963652028312D38293A2093
:105CB000000D0A496E76616C696420696E707574B6
:105CC000207265636569766564202D20496E707564
:105CD000742069676E6F7265642E0D0A5072657369
:105CE0007320616E79206B657920746F20636F6E0D
:105CF00074696E75652E2E2E0D0A001B5B324A00EC
:105D0000DACFE4FFE2CFDAFFE9CFE4FFEACFE4FF46
:105D1000F6CFE4FFF7CFE4FFF5CFE4FFF3CFE4FFE6
:105D2000F4CFE4FFFACFE4FF00EE00F0100EE80439
:105D300003E3EECFE4FFFBD700EE10F0080EE8041B
:105D400003E3EECFE4FFFBD7E652F2A414D09E0E9D
:105D5000D76E580ED66E0301642B000E65236623A2
:105D6000672303016A0706E1640E6A6F0301682B6B
:105D7000000E6923F2949E50200B05E09D50200BED
:105D800002E04EEC32F09E50100B05E09D50100BDF
:105D900002E064EC32F0E55200EE17F0080EE80481
:105DA00003E3E5CFEDFFFBD700EE0FF0100EE804A4
:105DB00003E3E5CFEDFFFBD7E5CFFAFFE5CFF4FF37
:105DC000E5CFF3FFE5CFF5FFE5CFF7FFE5CFF6FF32
:105DD000E5CFEAFFE5CFE9FFE5CFDAFF110088D88C
:105DE000B2EC34F0AFEC22F0F3EC0EF03AEC32F01F
:105DF00076EC31F0B2EC31F043EC32F001EC32F001
:105E000018EC32F02DEC32F00201140ED66F94EC47
:105E100031F00001F36FE0EC1DF044EC2AF05EEC91
:105E20000AF05CEC20F00201160ED66F94EC31F013
:105E3000010B06E10001010EFE6F0301070E756FF5
:105E40000201150ED66F94EC31F0020B0CE000014C
:105E5000FF510301645D106E320E105C04E364C3F5
:105E6000FFF0939C8A7C4FEC2AF0FEEC0AF06BEC7E
:105E700020F008D80001FE510301785DE1E078C30D
:105E8000FEF0DED703016C2B0C0E6C5D01E36C6B36
:105E9000C11C0F0B6C5D0FE2C30EC2166C51040DDA
:105EA000F350C212C280C282C2B2FED703012AD806
:105EB000C4CFEFFF120026D8EF6A1200350E0201A0
:105EC000F06FF16B6DC3EEF26EC3EFF2DBEC25F019
:105ED00000090DE13E0E0201F06FF16B6FC3EEF2AF
:105EE00070C3EFF2DBEC25F0000901E1010C000CBE
:105EF000040ED36ED3A6FED7D382F18ED56AF28E6E
:105F0000F28C12006C51EA6ACA0FE96E020EEA22A4
:025F100012007D
:0E5F12003DC373F30301726B0301080E716F40
:105F20006AEF34F03FC3AFFB40C3B0FBC750040B74
:105F300001E0010EE5D8FAE1C580C5B0FED7A1B6F3
:105F4000010C3EC374F3E1D801E0010CC750040B0F
:105F500001E0010ED5D8FAE1C5BC19D0B0CB74F37D
:105F6000D4D801E0010CC750040B01E0010EC8D8E1
:105F7000FAE1AFCB74F3C9D801E0010CC750040BB0
:105F800001E0010EBDD8FAE1C5AC000C020C020C18
:105F900042C33FF343C340F341C33EF3C3DF0B01AE
:105FA000086FE85005E178D80B01086FE85002E06F
:105FB00008511200C750040B01E0010EA1D8FAE10C
:105FC000C580C5B0FED7A1B6010C0301412903016C
:105FD000746F9BD801E0010CC750040B01E0010E67
:105FE0008FD8FAE1C5AC000C020CC750040B01E0DD
:105FF000010E86D8FAE144C374F387D801E0010C9E
:10600000C750040B01E0010E7BD8FAE1C5AC000CCF
:10601000020CC750040B01E0010E72D8FAE1C584EE
:10602000C5B4FED7000C79EC34F0C5B6FED7C59ADE
:10603000C588C5B8FED7C950120079EC34F0C5B692
:10604000FED7C58AC588C5B8FED7C584C5B4FED7F6
:10605000000C46C342F347C343F345C341F398DF03
:106060000B01006FE85016E103014A514A0700098D
:106070000EE0D9DFE66E030148C3E9FF49C3EAFF3A
:10608000482B000E4923E552E750EF6EEDD7D5DFE0
:106090000B01006F00511200C750040B01E0010E0C
:1060A0002FD8FAE1C584C5B4FED7A1B6010C000C07
:1060B000C750040B01E0010E23D8FAE1C580C5B03A
:1060C000FED7A1B6010C4BC374F31FD801E0010C3D
:1060D000C750040B01E0010E13D8FAE1A1B6010C80
:1060E000C5BC03D00B01B36B03D00B01040EB36F1F
:1060F000C584C5B4FED7A1B6010C0B01B351120083
:10610000106E1F0EC514101012007EEC34F0000942
:0261100012007B
:0E611200FB0EE3CFF6FFFC0EE3CFF7FFFD0E12
:10612000E3CFF8FFFE0EE3CFE9FFFF0EE3CFEAFF78
:10613000F90EE35003E1FA0EE35009E0F90EE3062D
:1061400002E2FA0EE3060900F550EE5CF1E01200FF
:10615000D9CFE6FFDACFE6FFFA0EE3CFD9FFFB0E89
:10616000E3CFDAFFFC0EE3CFE9FFFD0EE3CFEAFF5A
:10617000E9CFF3FFEACFF4FFF80EE35003E1F90EA5
:10618000E35008E0F80EE30602E2F90EE306DECF84
:10619000EEFFF2D7FF0EE3CFDAFFE552FF0EE3CFBB
:1061A000D9FFE5521200FB0EE3CFF6FFFC0EE3CF62
:1061B000F7FFFD0EE3CFF8FFFE0EE3CFE9FFFF0E82
:1061C000E3CFEAFFE9CFF3FFEACFF4FFF90EE350A4
:1061D00003E1FA0EE35009E0F90EE30602E2FA0EDB
:1061E000E3060900F5CFEEFFF1D71200FB0EE3CF77
:1061F000F6FFFC0EE3CFF7FFFD0EE3CFF8FFFE0E38
:10620000E3CFE9FFFF0EE3CFEAFF0900F550EF5CB3
:1062100002E1EE66FAD71200FB0EE3CFF6FFFC0EAA
:10622000E3CFF7FFFD0EE3CFF8FFFE0EE3CFE9FF6C
:10623000FF0EE3CFEAFFE9CFF3FFEACFF4FF090057
:10624000F5CFEFFFEE66FBD71200FE0EE3CFE9FFBE
:10625000FF0EE3CFEAFFF36AF46AEE5203E0F34A7B
:10626000F42AFBD71200D9CFE6FFDACFE6FFFA0E09
:10627000E3CFD9FFFB0EE3CFDAFFFC0EE3CFE9FF5C
:10628000FD0EE3CFEAFFE9CFF3FFEACFF4FFF80E0C
:10629000E35003E1F90EE3500BE0F80EE30602E2EF
:1062A000F90EE306DECFEFFFEE66F1D7DD52EFD752
:1062B000FF0EE3CFDAFFE552FF0EE3CFD9FFE55241
:1062C0001200FE0EE3CFE9FFFF0EE3CFEAFFE9CFB6
:1062D000F3FFEACFF4FF610EEF5C05E67B0EEF5CA7
:0C62E00002E7DF0EEF16EE52F6E11200AE
:0462EC00AA6AA96A87
:1062F0003F0EA6160B01B80E006F020E016FA950DB
:10630000106E116A120E105C000E11580CE2A6807D
:1063100000CBE9FF01CBEAFF002B000E0123A8CF41
:10632000EFFFA92AECD71200D6C2A9FFAA6AA6B22B
:10633000FED73F0EA616A680A8501200D7C2A9FF0E
:10634000AA6AA6B2FED72F0EA616A684550EA76E71
:10635000AA0EA76EA6820000A6B2FED7A69400D011
:1063600012001200240EAC6E900EAB6E080E7E6E04
:1063700002011F0E7CD8080A36E00F0A32E0010A3B
:106380002AE0030A23E0010A1CE0070A15E0010ADB
:106390000EE0030A07E0010A28E10B01340E1C6F2E
:1063A000820E1DD00B018C0E1C6F200E18D00B011D
:1063B000450E1C6F100E13D00B01220E1C6F080E21
:1063C0000ED00B01100E1C6F040E09D00B01080E2D
:1063D0001C6F020E04D00B01030E1C6F010E1D6F0B
:1063E00008D0AC0E03D0560E01D0AC0E0B011C6FC2
:1063F0001D6B1CCBAFFF1DCB10F0116A10507F6ED0
:1064000012000201230E33D8926E0201240E2FD8FF
:10641000936E0201250E2BD8D809946E0201280E26
:1064200026D8976E0201290E22D81009986E120004
:1064300002012A0E1CD8896E02012B0E18D88A6E12
:1064400002012C0E14D88B6E02012F0E10D88E6E06
:106450000201300E0CD88F6E12000201310E07D8E7
:10646000C16E0201320E03D87F0BC06E1200D66FD0
:0464700094EF31F084
:0C6474000001EC6BE06BE16BEA6BEB6B82
:106480009D9A9D9812009D8A9D9812000001E16BD3
:10649000E1C0E0F0EB6BEBC0EAF01200060EAB14CB
:1064A00002E0AB98AB889EAA0ED00001EB51EA6ADD
:1064B000E20FE96E000EEA22AECFEFFFEB2B070EE4
:1064C000EB15EB6FF0D712000001E051E15D0DE03C
:1064D000E051EA6A600FE96E000EEA22EF50AD6EFD
:1064E000E02B7F0EE015E06F12009D981200120065
:1064F0000001EC5112000001EA51EA6AE20FE96E74
:10650000000EEA22EFCFAFFBEA2B070EEA15EA6F87
:106510000B01AF5112000001E129106E116A7F0ECC
:106520001016000E11160001E051126E136A12507F
:10653000101802E11350111802E10400ECD7F29E8A
:106540009DB805D0EDC0ADFF9D88F28E11D0000141
:10655000E151EA6A600FE96E000EEA22EDC0EFFF3A
:106560000001E12B7F0E0001E1150001E16FF28EC9
:1065700012000001EE519F0805E2EE390F0B0F0BE0
:10658000570F04D0EE390F0B0F0B300F0001ED6FDA
:10659000C2DF0F0E0001EE15090804E20F0EEE1522
:1065A000570F03D00F0EEE15300F0001ED6F8BEF7C
:1065B00032F00001EFC0E9FFF0C0EAFFEF2B000E60
:1065C000F023EFCF08FBEF5004E008CBEDF0A3DFA2
:1065D000F0D712000001F1C0F6FFF2C0F7FFF12B77
:1065E000000EF2230800F5CF00FBF55004E000CBCD
:0865F000EDF091DFEFD712007E
:0865F8000D01EF6BF069F16980
:10660000F269F369F469F569F66BF76BF86BF96B8E
:1066100012000D01EF5129E10301260E5D6F0B0EF3
:106620005E6F03011C0E5B6F0B0E5C6F00EC29F0BC
:1066300000092CE00B01265115E11CCBF0FD1DCB10
:10664000F1FD1ECBF2FD1FCBF3FD20CBF4FD21CBE2
:10665000F5FD22CBF6FD23CBF7FD24CBF8FD25CBB2
:10666000F9FD010C0D01010EEF6F34EC14F000097F
:106670000CE00301616B03011C0E5F6F0B0E606F7A
:1066800073EC29F00D01EF6B010C000C010CFACD3D
:10669000E9FFFBCDEAFFEECF22FBEECF23FBEECFEF
:1066A00024FBEFCF25FB0301010E616F03011C0EDC
:1066B0005F6F0B0E606F73EF29F0FCCDE9FFFDCD2E
:1066C000EAFF0D01F651EE1808E1F751EE1805E169
:1066D000F851EE1802E1F951EE1814E00201C6512A
:1066E0000D01F65D20E10201C7510D01F75D1BE1CF
:1066F0000201C8510D01F85D16E10201C9510D01F9
:10670000F95D11E1FECDE9FFFFCDEAFFF0CDEEFF2F
:10671000F1CDEEFFF2CDEEFFF3CDEEFFF4CDEEFFC7
:08672000F5CDEEFF010C000CA9
:086728005458540048544D0080
:10673000434C4100435353004A530000474946002D
:10674000434749004A5047004A41520057415600CA
:10675000545854005A5458005A4854005A434C0054
:106760005A4353005A4A5300485454502F312E3044
:1067700020323030204F4B00436F6E74656E742DA5
:10678000747970653A2000436F6E74656E742D45A0
:106790006E636F64696E673A20677A69700D0A00EC
:1067A000457870697265733A20300D0A0043616361
:1067B00068652D436F6E74726F6C3A206D61782D31
:1067C0006167653D3330302C206D7573742D7265B3
:1067D00076616C69646174650D0A0047455400492F
:1067E0004E4445582E48544D004C4F47494E2E4379
:0367F00047490016
:0C67F4002A0EF66E000EF76E000EF86E16
:1068000002010900F550FB6F0900F550FC6F03E130
:10681000FB6701D03DD00900F550F66F0900F55037
:10682000F76F0900F550F86F09000900F550E96E9F
:106830000900F550EA6E090009000900F550F96FEA
:106840000900F550FA6F09000900F6CFFDF2F7CF05
:10685000FEF2F8CFFFF2F6C2F6FFF7C2F7FFF8C27A
:10686000F8FF0201F95302E1FA5307E00900F5507D
:10687000EE6EF907F8E2FA07F9D7FDC2F6FFFEC29D
:10688000F7FFFFC2F8FF0201FB07000EFC5BBFD75A
:026890001200F4
:0E6892004E6F7420496D706C656D656E746597
:1068A000640073656C656374656400636865636B3D
:1068B00065640064697361626C6564003C212D2D20
:1068C000002D2D3E006F6E006F666600557064618E
:0368D000746500EC
:0C68D4003F0EC716C66AC56A0301715169
:1068E000C6127251C71294869488C68A73C3C8FFB1
:1068F0001200C586C7A0FED7C950120074C3C9FFD5
:0A690000C6BEFF0CC7B0FED7000CA6
:06690A00FF0EE3501D6EBC
:10691000EF0E01D0F30EE76EE72E8CEF34F00C0E85
:106920001C6EE76AE72E92EF34F01C2E91EF34F0E4
:086930001D2E8AEF34F0120065
:08693800036A026A100EE76E0B
:10694000D89006360736023603360B50025C0C50E0
:10695000035805E30B50025E0C50035A062AE72E3B
:04696000F0D712005A
:0C6964000301646B656B666B676B686B0E
:10697000696B580ED66E9E0ED76E010ED56ED58EF3
:06698000F284F28A12000D
:0A698600036A080EE76ED89007368A
:1069900003360C50035C02E3036E072AE72EF7D799
:0269A0001200E3
:0E69A2001EEE00F02EEE00F0F86A0F9CFAECEC
:0A69B00033F0EFEC2EF0FDD71200DB
:0669BA00FF0EE350E84E61
:1069C0001200000000D000D000D0E82EFAD712004C
:0669D00056322E343300A4
:0669D60056332E303400A0
:0469DC0018510151FC
:0C69E000E550CD50AD508C504D50305063
:0269EC000000A9
:0269EE000000A7
:1069F00011500750F34FEA4FDA4FD04F0750C54FB1
:106A0000AC4F9F4F115011500750F34FEA4FDA4FE0
:086A1000784F584F534F2C4FF3
:086A1800FB51F651F151EC5164
:106A2000E751E251D651BE51AE51A4519D5187510B
:0A6A3000725157514B5133512A5156
:046A3A0000FF000059
:020000040030CA
:0100010026D8
:0100020004F9
:010003000AF2
:010005008377
:010006008178
:010008000FE8
:01000900C036
:01000A000FE6
:01000B00E014
:01000C000FE4
:01000D0040B2
:0200000400F00A
:100000000A0100010004A3000000FF0000000A0133
:10001000000104012803000A0100010A0100010790
:10002000000700FFFFFFFFFFFFFF000000000000D0
:1000300000032E000061646D696E0000000070779F
:0700400000000000000000B9
:00000001FF
